:020000040000fa
:08000000e40804000000000008
:020000040000fa
:10040000889fbe008a9fbe00010578000100e000c1
:100410000400350008003c000000e000200032002d
:100420000500370060001000e080180002003b006b
:1004300001f02c001a0037000004be006011b80063
:100440006b0920000982cf00020039000882cf002a
:100450000441b000694252000e00320008003b0027
:1004600082817100610164008904d1000884d30095
:100470008b05e8000442e800f9ff3a000500370068
:100480000804440089844c008b05e9000442e9001b
:10049000fbff3a00540107000af0a70001f0a0009a
:1004a0004f05be004f04be0000000600889fbe003e
:1004b0008a9fbe008c1f780071010700780133000d
:1004c00003866c006450e100240032006420e100e7
:1004d000270032006150e100220032006120e1007b
:1004e000210032008b854200eb07b1000134b800d7
:1004f000003ab8000804420089844a00013ab80072
:100500000030b8008880400009014a000400330030
:100510000000400081804800020149008b05e9008d
:10052000c909dd00830170000100320013002000c2
:10053000c814de004814dd004709de001200b200d6
:10054000c808de00088470002701070001f0a10040
:100550000cf0a70001f0a0005a0137006120e10073
:100560005c0132000801be000200be00f7ff370048
:100570006150e100fcff3a0056013700889fbe0041
:100580008a9fbe008c1f78003d01070044013300a4
:1005900003866c006450e1002e0032006420e1000c
:1005a000330032006150e1002f0032006120e10091
:1005b0003100320085855500eb07b00009002000ae
:1005c00008042000050037000804440089844c001a
:1005d0000a0031000603430087834b0000015300eb
:1005e00081815b00f8ff33000203be000800a00019
:1005f0000804440089844c00f6ff3900c639dd0048
:100600008301730001003200130020008904d1002f
:100610000884d3000998a300050032000800a70051
:100620000300a0008904d1000884d3008b05e800f2
:100630008904d1000884d3000001eb000281d200bc
:10064000e900070001f0a1000cf0a70001f0a000f4
:100650001c0137006420e1001e0132000801be00c9
:100660000200be00f7ff37006120e10019013200ef
:100670006000b800f3ff37000000200001f82700f9
:10068000f0ff370003f0a200889fbe008a9fbe00e3
:100690008c1f7800fa000700010133006450e1006c
:1006a0004f0032006420e1005200320003826c00ef
:1006b00007003b000905d0000306d000820f54005c
:1006c0000c065d000200390002003200890178004a
:1006d000030678008582550004003d000003fd00fc
:1006e0008103fd008502ea008b854200840f7200c1
:1006f00002003b0060001000e08018006011b800ac
:100700000005eb007a28e1000a00390006007800b5
:10071000c75ddd00f707b200878075002d00370048
:10072000828171000a017800610560008180d1003a
:100730000080d3008502e900f9ff3b000604400079
:100740008784480002003b0060041400e0841c0021
:100750000988a300070032008a817100828171003c
:10076000610164008904d1000884d3008b05e8008e
:10077000170037000978a30013003a000b00e000cf
:10078000130034008b05e9000804440089844c0000
:100790000a4474000978a3000d003a000b00e00041
:1007a000070034008b05e9000804440089844c00ec
:1007b00001003a000b0020000978a300f7ff320087
:1007c0000001eb0002003700828171000a0178000d
:1007d000850007000cf0a70001f0a000b900370069
:1007e0006420e10002003a00838f6c00b9003300fe
:1007f0000801be000200be00b20037000001be00ca
:10080000b70007000470a70003f0a1006509b1005c
:10081000160032000d0035006828e10006003500a2
:10082000f0ff2f00f1ff27000300e00013003b0062
:100830000100280000000500000040008180480001
:100840008502e900fcff3a0008003700f88f4200fb
:1008500002003c008000eb00000005008100d10098
:100860000080d3008502e800fcff3a000300e000ae
:1008700002003b0060001000e0801800000006004d
:10088000889fbe008a9fbe008c1f78007c000700f6
:100890001002200002003b0000408800800037006a
:1008a0008a0062006408e10002003a00004088000b
:1008b000880037006108e100fcff32000800be003c
:1008c000030478002dff070001f0a1009900070044
:1008d00008f0a600040037000001be0091042400c7
:1008e000b0fd200067ff070009f0a70001f0a2009b
:1008f00074003700889fbe008a9fbe008c1f78005e
:100900000004be00760007000478a30026003a0029
:100910006120e1002500320009f8a30025003a001b
:100920006420e10021003200f507b1000508a300b2
:100930000200320000004000818048006044b8009e
:1009400003102000020020000000400081804800c9
:100950000805440089854c000a0541008b85490043
:100960000a0550008b855800030033000a00be00c2
:1009700002047400838474008301d1000281d300d7
:10098000830f7100f0ff3a008904d1000884d3007e
:100990006001490082017800c1adde00fb07b000b4
:1009a00011000700470037000960a0000800be00e2
:1009b000440037001202200002408800f0ff2f00a0
:1009c000f1ff27003f0037000001eb00be003700b9
:1009d0000081eb00bc0037000001eb002301370071
:1009e0003200200021013700810020006180550085
:1009f0000b003d000b00200061fe2f000100e10014
:100a00001d00340082817100610164008904d100fd
:100a10000884d3000000e800faff3a0071002000cb
:100a200061006400030070000200600009003200f1
:100a300061044400e0844c000988a50005003200f0
:100a40008b05e8006808e10002003a008904d10043
:100a50000884d300f20f20000258e10005003d0099
:100a6000c75ddd00f907b2008980750008007800d5
:100a7000000006000bf827008b007800000005003e
:100a80000004be00160007000003be000405be00ff
:100a90000200be0012000700844f7500000006002f
:100aa0000200be006450e100050036006420e10051
:100ab000020036000968a30001003a000800be00e9
:100ac0000160a0004f0678004f05be004f04be0035
:100ad00000000600f0ff2f00f1ff2700f9ff3700ac
:100ae000c70ade00f107b200f50fb20008003200bd
:100af000e1cf4200020032000170a0002400050096
:100b0000810f700001003200040805004400050058
:100b1000810f700002003a00140005008502e90010
:100b20000000400081c04800fcff3b000170a000b5
:100b300024000500889fbe008a9fbe008c9fbe00d7
:100b40000004be00e6ff07000800be00890678002a
:100b50006420e10008003900040032000160a000b8
:100b600012022000024088005300370091fc23004d
:100b7000b0fd20004e0037000006eb0009f0a10098
:100b800003f82300020020000800be001e01070039
:100b90000600340001f82300000020000801be0018
:100ba00076fe07000004be002c0020000800be00f6
:100bb00093e82300320a23001301070012003400d7
:100bc0000801be00d1fd2300703d2b00aefe0700e2
:100bd0000005be00b3f32300f27a26000800be0031
:100be00032fe070003f8230002002000a5fe0700e4
:100bf0000801be00a4fe07000a01be005ffe070058
:100c00000004be000c06e8000800be0001f0a100d0
:100c10000200200003982300fb0007000800be002c
:100c2000160035000801be0020fe07000005be00ca
:100c300032cd2c0043fb230093fe0700809fbe00b3
:100c40001269280003d52b000a00be0017fe07001a
:100c5000620f210013ef2b008bfe07000a01be007c
:100c600012fe07004f01be0044fe07000801be004f
:100c70000efe07000801be0083fe07000c00e00026
:100c80000b0032000c10a70001f0a200b2fd200002
:100c900093fc23006260e1000400320022a92000de
:100ca00063f023000c10a70063f8230076fe070012
:100cb0000df0a70001f0a2004f06be004f05be00d8
:100cc0004f04be0000000600889fbe008a9fbe0041
:100cd0008c9fbe00820578000004be0080ff0700e4
:100ce0000800be006420e1000700390002003a005d
:100cf000f1ff2700f0ff2f000160a000120220008a
:100d000002408800550037006120e10003003a00ee
:100d10000b00a70001f823005000370001f0a100ec
:100d20000200210093642400b70007000800be0001
:100d300004003500b2fd2000930c2400b40007002d
:100d40000004be000005eb000b00a6004f0dde0006
:100d500001f0a1000004be0032982f0023ea230016
:100d6000d2fd07000001eb0003f023000b00a700f9
:100d700003f8230044fe0700a0fe07000000a700c0
:100d80000a00a2009efd07000b00e00003003200f5
:100d90000200200003f023003afe070001f0a20049
:100da0000006be000200200093042400bffd0700df
:100db0000801be0034fe0700809fbe000c00be008c
:100dc00022a22a00d3a72300b8fd07004f01be00ce
:100dd0002dfe07000004be0001f0a100020020006b
:100de00003982300880007000800be0019003500a2
:100df0000001be00adfd07000006be00b2c529001f
:100e0000e3622300a9fd070022222b00f3942b00ac
:100e10001dfe07000c01be00a4fd0700e2732800c0
:100e200083c0230018fe07000c01be009ffd0700d1
:100e300042aa2a00a3e22b0013fe07000c01be0009
:100e40009afd07000801be0098fd07000801be00da
:100e50000dfe07000a00a70001f0a2004f06be0029
:100e60004f05be004f04be0000000600889fbe0074
:100e70008a9fbe008c9fbe000206780001f0a7008a
:100e80000cf0a0000004be0015ff07000800be0023
:100e90006420e1000700390002003a00f1ff27005a
:100ea000f0ff2f000160a000120220000240880025
:100eb0005100370009f0a1000800be000200200028
:100ec00003f8230054000700f4ff3c000800be00b4
:100ed00002002000039823004b0007000800be001a
:100ee000300035000200200003f023004a00070014
:100ef00005003c000800be000801be006bfd0700b5
:100f00000005be000e0037000c10a20000002000fb
:100f100001f823000801be00dafd070002002000ee
:100f200003f0230061fd07000005be0071fe07000d
:100f30000200200003002c005cfd07000004be003e
:100f40000a00be00b2d02800130b2c00cefd070013
:100f50000a01be0055fd0700020f2500330b2400d7
:100f6000c9fd0700809fbe000a00be005206220095
:100f700013f02b004dfd0700b2662100f3f62300ad
:100f8000c1fd07000a01be0048fd07004f01be0079
:100f90007afd07000801be0044fd07000801be00fd
:100fa000b9fd07000c00a70007003700b2fd2000c4
:100fb00093fc23000c10a700b3fd07000cf0a70062
:100fc00001f0a2000c0037000cf0a700020037006f
:100fd00001f0a20004003700b2fd200093042400b9
:100fe0000c10a60003003700b2fd200093fc230084
:100ff0000c10a700a4fd07004f06be004f05be0061
:101000004f04be000000060014002000040037005a
:10101000040020001d003700f4ff2f0000003700ff
:10102000889fbe008a9fbe00841f780094fe070040
:101030004f00780011003300f0ff2f00838f6c0009
:1010400006003b00040565000a00a7000800370001
:1010500009f0a6001000200008003700820f54009d
:10106000838f5c00030039001000200001003e0067
:101070000000200009f0a7000000ea004f05be00b4
:101080004f04be000000e00000000600889fbe0084
:101090008a9fbe008c1f78004f26dd0078fe070077
:1010a0007ffe33006120e100430032006250e10026
:1010b00041003e003e0039006420e1003c00320067
:1010c000058255000f003b000402e80038003a009a
:1010d000800f5300818f5b00350034000800be0094
:1010e00003f0a10001f0a60003f0a0000cf0a7009f
:1010f00065fd070073fe37000603430087834b003e
:101100000c4646000005530081855b000200330059
:101110000a03be000c00a0000402e900f6ff3b0039
:10112000850578000602430087824b0004003a00e0
:101130006000b80009f0a70001f0a00061fe3700d0
:101140000002520081825a000704e00004003300cc
:101150000603430087834b008b05e900faff370045
:10116000090578000604be000203be006011b80045
:101170001dfe0700e00f5200e08f5a000700350007
:1011800002003c000c08a300040032000601be006f
:1011900003f0a0000cf0a7003bfd07000a856800e3
:1011a00001f0a1000af0a70001f0a00045fe370001
:1011b0000800be0043fe3700100220000cf0a6001d
:0811c0000040880043fe3700e7
:020000040000fa
:0200000401f009
:04000800fdff0000f8
:020000040000fa
:0200000401f009
:04000c0078ff000079
:020000040000fa
:0200000401f009
:040010007dff000070
:020000040000fa
:0200000401f009
:04001400e7ff000002
:020000040000fa
:0200000401f009
:04001800fcff0000e9
:020000040000fa
:10000800b4420000b4420000b4420000b442000010
:10001800b4420000b4420000b4420000b442000000
:10002800f2330000523c00007e3e0000b442000063
:10003800b44200008e3c00008a3e0000a63e00004c
:10004800b4420000b4420000b4420000b4420000d0
:10005800b4420000b4420000ee3e0000b44200008a
:10006800b4420000b4420000b4420000b4420000b0
:10007800b4420000b4420000b4420000b4420000a0
:10008800b4420000963e0000a23e0000b4420000c8
:1000980064310000b4420000ce300000b4420000d9
:1000a800b4420000b4420000b4420000b442000070
:1000b800b4420000ca3c0000263d0000623d00003a
:1000c800da3d0000b4420000b4420000b44200002f
:1000d800b4420000b4420000b4420000e03e000018
:1000e800c23e0000b4420000b4420000b442000026
:1000f800b4420000b4420000b4420000b442000020
:10010800b4420000b4420000b4420000b44200000f
:10011800b4420000b4420000b4420000b4420000ff
:10012800b4420000b4420000b4420000b4420000ef
:10013800b4420000b4420000b4420000b4420000df
:10014800b4420000b4420000b4420000b4420000cf
:10015800b4420000b4420000b4420000b4420000bf
:10016800b4420000b4420000b4420000b4420000af
:10017800b4420000b4420000b4420000b44200009f
:10018800b4420000b4420000b4420000b44200008f
:10019800b4420000b4420000b4420000b44200007f
:1001a800b4420000b4420000b4420000b44200006f
:1001b800b4420000b4420000b4420000b44200005f
:1001c800b4420000b4420000b4420000b44200004f
:1001d800b4420000b4420000b4420000b44200003f
:1001e800b4420000b4420000b4420000b44200002f
:0801f800b4420000b442000013
:020000040000fa
:10020800b4420000b4420000b4420000b44200000e
:10021800b4420000b4420000b4420000b4420000fe
:10022800f2330000523c00007e3e0000b442000061
:10023800b44200008e3c00008a3e0000a63e00004a
:10024800b4420000b4420000b4420000b4420000ce
:10025800b4420000b4420000ee3e0000b442000088
:10026800b4420000b4420000b4420000b4420000ae
:10027800b4420000b4420000b4420000b44200009e
:10028800b4420000963e0000a23e0000b4420000c6
:1002980064310000b4420000ce300000b4420000d7
:1002a800b4420000b4420000b4420000b44200006e
:1002b800b4420000ca3c0000263d0000623d000038
:1002c800da3d0000b4420000b4420000b44200002d
:1002d800b4420000b4420000b4420000e03e000016
:1002e800c23e0000b4420000b4420000b442000024
:1002f800b4420000b4420000b4420000b44200001e
:10030800b4420000b4420000b4420000b44200000d
:10031800b4420000b4420000b4420000b4420000fd
:10032800b4420000b4420000b4420000b4420000ed
:10033800b4420000b4420000b4420000b4420000dd
:10034800b4420000b4420000b4420000b4420000cd
:10035800b4420000b4420000b4420000b4420000bd
:10036800b4420000b4420000b4420000b4420000ad
:10037800b4420000b4420000b4420000b44200009d
:10038800b4420000b4420000b4420000b44200008d
:10039800b4420000b4420000b4420000b44200007d
:1003a800b4420000b4420000b4420000b44200006d
:1003b800b4420000b4420000b4420000b44200005d
:1003c800b4420000b4420000b4420000b44200004d
:1003d800b4420000b4420000b4420000b44200003d
:1003e800b4420000b4420000b4420000b44200002d
:0803f800b4420000b442000011
:020000040000fa
:1088000000800000000000000f0000002d000000ac
:1088100001000000160000000000000069000000d8
:10882000460000008200000000000000010000007f
:1088300004000000070000000b0000000e00000014
:1088400004000000070000000b0000000e00000004
:10885000000000000100000004000000070000000c
:108860000b0000000e0000000400000007000000e4
:108870000b0000000e0000000000000001000000de
:1088800004000000070000000b0000000e000000c4
:1088900004000000070000000b0000000e000000b4
:1088a00000000000010000000400000007000000bc
:1088b0000b0000000e000000040000000700000094
:1088c0000b0000000e00000000000000010000008e
:1088d00004000000070000000b0000000e00000074
:1088e00004000000070000000b0000000e00000064
:1088f000000000000100000004000000070000006c
:020000040000fa
:109000000000000000000000050000000a00000051
:1090100002000000160000000000000069000000cf
:1090200064000000780000000a000000aa030000ad
:10903000aa0300002c030000aa0300007d0000002a
:1090400040000000140000000000000000000000cc
:10905000aa030000000000000a00000064000000f5
:10906000190000000000000000000000aa0300003a
:10907000aa0300002c0300001400000005000000fb
:10908000010000001f07000047070000490700001b
:109090002005000052000000560000005b000000a8
:1090a0004f000000530000004400000000000000da
:1090b00000000000000000000000000000000000b0
:1090c000020000000200000000000000000000009c
:1090d000000000000000000000000000ffff000092
:020000040000fa
:1011c8008fef2000007f240000018800000000004d
:1011d800560f020000000000e0012000303a8800ad
:1011e80044e7a90044c7a9004487a9004467a900a7
:1011f8004447a9004427a9004407a900300020005b
:101208003174200082072000a3092000824878005a
:10121800834878008048780010002000217420005e
:101228006204200073052000824878008348780013
:10123800804878002aa3ef002c23ef002023ef003a
:1012480021e3a90021a3a8002183a8002143a80025
:101258002123a9002103a90020e3a80020c3a80096
:1012680020a3a8002063a9002043a9002023a900e7
:1012780023e3a90023c3a90023a3a9002383a9006a
:101288002343a8002323a9002303a90022a3a8001d
:101298002283a9002263a8002243a8002223a900d0
:1012a8002203a900f0f12100201988003223ef0061
:1012b8002623ef002823ef0029e3a90028e3a9004b
:1012c8002963a9002943a9002923a9002903a90002
:1012d8002863a9002843a9002823a9002803a900f6
:1012e8002e23ef00f0ff200080198800aa80a900b3
:1012f800aaa0a900aac0a9008ca3a9008c83a90050
:101308008c23a8008c03a900d0c0b300701c8800ef
:101318009023ef00c0022000901c880000302000bd
:10132800a01c8800b0002000b01c8800ab40a900b9
:10133800ab20a900ab00a90085c0a90000002000cf
:10134800401188002222ef0023e2a90023a2a9006d
:101358002022ef002042a8002022a9009580a900a1
:101368009560a90030102000c011880033e2a90060
:1013780033a2a900b340a800b320a900b300a90074
:101388003022ef003042a9003022a90032e2a90041
:1013980032c2a90097e0a90097c0a900a4c0a8007c
:1013a800a4a0a900a480a8004221ef0010082000f2
:1013b800100a8800a6c0a800a6a0a900a680a800b8
:1013c8004621ef0010082000300a8800b6c0a800a7
:1013d800b6a0a900b680a8004a21ef001008200096
:1013e800500a8800b740a800b720a900b700a80095
:1013f8004e21ef0010082000700a8800b7c0a8002e
:10140800b7a0a900b780a8005221ef00100820005b
:10141800900a8800b840a800b820a900b800a80021
:101428005621ef0020002000b00a8800a540a8003f
:10143800a520a800a500a9008421ef00a740a800c6
:10144800a720a800a700a9008a21ef00b0c0a80023
:10145800b0a0a800b080a9009021ef00b140a8007a
:10146800b120a800b100a9009621ef000622ef00e4
:101478000822ef00ca22ef00d022ef00d622ef00a8
:10148800e222ef00c6a2ef00cca2ef00d2a2ef004a
:10149800dea2ef00cdc2a900cda2a900d202a90008
:1014a800d222a900d242a900d262a900de02a90074
:1014b800de22a9001e21ef002021ef001421ef00f9
:1014c8001821ef0030002000e008880000d4200038
:1014d800d00888001e61a800b240a900b220a80068
:1014e800b200a8008780a9009780a8001021ef000b
:1014f8000621ef00400d23006008880010a1a80015
:1015080084e0a90094e0a800a7c0a800a7a0a800ac
:10151800a780a9001221ef000a21ef00f0ff2f0099
:10152800700888001281a8002c21ef002221ef000a
:1015380090d02300400988002c81a8002ca1a80085
:10154800bbc0a800bba0a800bb80a90089e0a90077
:1015580099e0a8002e21ef002621ef0090d023006b
:10156800500988002ea1a8002e81a800bc40a80020
:10157800bc20a800bc00a9008a00a9009a00a80005
:10158800a440a900a420a800a400a9008200a900e2
:101598008400a9009400a8000421ef000021ef00b6
:1015a80005e1a900fc0c020000000000704f2400b7
:1015b800d05b880000002e00e05b8800704f24009c
:1015c800f05b880000002e00005c8800704f24004b
:1015d8008048880000002e009048880021e2a8007a
:1015e800f00c02000000000080cd20007060880030
:1015f8008560a90021e2a80087c0a90097c0a800bb
:1016080031e2a8008900a9009900a8008420a90057
:101618009420a80084a0a90094a0a80088a0a900ec
:1016280098a0a80088c0a90098c0a80088e0a900d0
:1016380098e0a8008440a9009440a80084c0a900ac
:1016480094c0a8008720a9009720a8008740a90077
:101658009740a800e202a900e222a90085a0a900fb
:1016680011e1a8002de1a800a03a20004049880017
:10167800100c8800407520005049880030a02000d8
:1016880060498800c0da200070498800609a20000c
:101698008000eb003c000800010000000118780001
:1016a8008100e800024002000000000056c9a800be
:1016b8000b08a9003a09a9003aa9a9003a69a900a2
:1016c8000c28ef000007200060418800004c8000d3
:1016d800030120000300b90043062000110009009f
:1016e8004308d80030568800704a80000301200063
:1016f8000300b90043062000110009004308d80080
:10170800f0558800804a8000030120000300b900da
:1017180043062000110009004308d800005688003d
:10172800904a8000030120000300b900430620000e
:10173800110009004308d80010568800a04a80000c
:10174800030120000300b90043062000110009002e
:101758004308d80020568800704b8000105188003c
:10176800030120000300b90043062000110009000e
:101778004308d800c0558800804b80000301200032
:101788000300b90043062000110009004308d800ef
:10179800e0558800904b8000030120000300b90049
:1017a80043062000110009004308d800d0558800de
:1017b800204d8000014d8000010050008000eb00aa
:1017c800000202000000000003482400020020007c
:1017d800be020200000000006148880070488800ce
:1017e800004b800040518800030120000300b9002d
:1017f80043062000110009004308d800b0558800ae
:101808008000eb00d04a80000002020000000000c7
:1018180091588800a05888008000eb00f04a8000aa
:101828000002020000000000d1588800e05888003b
:101838008000eb00404b8000000202000000000026
:10184800f1588800005988008000eb00604b800048
:101858000002020000000000315988004059880049
:101868008000eb00e04a8000000202000000000057
:10187800b1588800c05888008000eb00504b8000a9
:101888000002020000000000115988002059880059
:101898008000eb00304b80000002020000000000d6
:1018a80091558800a05588008000eb00204b8000ef
:1018b80000020200000000000312240002002000c1
:1018c8005602020000000000b15d8800c05d88007b
:1018d800914c8000804c8000000202000000000053
:1018e800a3c52400920e2900be02020000000000d9
:1018f8003152880020528800934c8000824c80002e
:10190800880e020000000000a1a5200060c0200091
:10191800a0107800a0107800a0107800a01078001f
:10192800a0107800a0107800a0107800a01078000f
:101938005e0aa900f20baf005e0aa800b14c800055
:10194800a04c80000002020000000000a3c5240093
:10195800920e2900be0202000000000051528800c9
:1019680040528800b34c8000a24c8000880e0200d0
:101978000000000001a7200060c02000a01078002f
:10198800a0107800a0107800a0107800a0107800af
:10199800a0107800a0107800a0107800a01078009f
:1019a800720aa900f20baf00720aa8003089a900d8
:1019b80062e9af003089a80030a9a9006309af0027
:1019c80030a9a80021e3a8008de3a8002043a800bf
:1019d80000000000feff3700e42aef00e22aef00d3
:1019e800e02aef001fe1a80013e1a80000000600ac
:1019f8002180200062ef20008018eb000208e6003a
:101a0800fdff370000000600c24780000290b900c1
:101a1800305f8800415f8800d24780000290b9009b
:101a2800e62bb40001007800e8abb400e247800080
:101a38000290b900e62bb40001007800e8abb400ce
:101a48003c0e020000000000305f8000b0578800a4
:101a580000000600c0478000d05e8800d2478000a2
:101a68000290b900305f8800415f8800e24780003b
:101a78000290b900e62bb40001007800e8abb4008e
:101a88003c0e020000000000305f8000c05e88004d
:101a9800e147800001f0a700d82bee00c05e80006f
:101aa8008000eb0000f0a7008080eb00000202003d
:101ab80000000000915c8800a05c8800d05e800077
:101ac8008000eb0000f0a7008080eb00000202001d
:101ad80000000000935c8000a25c800040040200cb
:101ae80000000000515a8800605a88000000060073
:101af800d0478000d05e8800c24780000290b900bd
:101b0800305f8800415f8800e24780000290b9009a
:101b1800e62bb40001007800e8abb4003c0e0200ec
:101b280000000000305f8000c05e8800e147800050
:101b380001f0a700d82bee00c05e80008000eb000b
:101b480000f0a7008080eb00000202000000000007
:101b5800915c8800a05c8800d05e80008000eb006b
:101b680000f0a7008080eb000002020000000000e7
:101b7800935c8000a25c800040040200000000002a
:101b8800715a8800805a880000000600d25e8000e2
:101b9800f30720000310b900c45e8000110009009b
:101ba8004408d800305f8800e7ebaf00e62bee0072
:101bb800f1032000e15e8800000020009001880009
:101bc800a00d2400e15e80004200a9008180d200bf
:101bd800008040009000ba00325f80000208e600f2
:101be80002003700dc2bed00f3ff3a00dc0be200cb
:101bf80018003200fde8ae0007003700dbebae004e
:101c08000c00370000082000e15e80000100400061
:101c1800f05e880000000600dbebae000a0037002b
:101c280000102000e15e800001005000f05e880096
:101c38000000060000082000e15e8000010050005e
:101c4800f05e880000000600e05e8000f05e88001c
:101c580000000600fde8af0002003700de2bef00b1
:101c68000000060000082000f05e88000000060062
:101c7800e88bd6004200af0000000600f20e02001a
:101c880000000000fc0e020000000000000120001f
:101c9800105f8800eeabd600f0abd600eaabd600fa
:101ca800ecabd600eeabd600f0abd600eaabd60074
:101cb800ecabd6004200a800e6abd600e8abd600f5
:101cc800405f8000ec0bb50002003a00305f8000f6
:101cd800ea0bb50005003900305f8000ea2bb5003b
:101ce800405f8000ecabb500e62ba800e60ba9002e
:101cf800e22bed00e7ff3a004200a900e8abd7006d
:101d0800e6abd70000000600e02bef00060f02004c
:101d1800000000004200af00000006003e0f020075
:101d28000000000000022000105f88000281d2003d
:101d38008381d20066c02000090008000600000068
:101d4800168bd200a000200096007800008050007a
:101d58004200af00000b780026007800e22bed006f
:101d6800f2ff3a00e00baf00f20ba8004200a90016
:101d780000000600005f880000022000105f880055
:101d880042bf2000a00020004200a900015f80009f
:101d980001800800020000004200af001209400064
:101da8001299d300e8abd700e6abd700e22bed00e1
:101db800f3ff3a0042007800f1ff2f000080400056
:101dc8004200ae00e88bd6004200af0000000600db
:101dd800f20baf000e00070000000600305f800025
:101de800705f8800405f8000805f88000000060008
:101df800ea2bef00ec2bef00e62bef00e82bef00cf
:101e0800000006000380d2004200ae000000060079
:101e1800405f80000100280001006000e6abee0092
:101e2800e8abee00e62bec0001003a00e82bec00f2
:101e3800e02bec00e80bb40000000600ec8bd600a9
:101e48004200ae0000000600605f8000010028002c
:101e580001006000eaabee00ecabee00ea2bec0010
:101e680001003a00ec2bec00e02bec00ec0bb4008a
:101e780000000600f22bef00f42bef00f62bef002a
:101e8800f82bef00fa2bef00fc2bef00fe2bef00f6
:101e9800002cef00022cef00042cef00062cef00c2
:101ea800000006000000eb00000778000c000900a5
:101eb800002f78000007eb0000000600c04c8000ef
:101ec800310020000180e700200037002041800019
:101ed800410620006329af00010040006329ae00dd
:101ee80001005000c14420000180e6006329a900d8
:101ef80041bb2f000100e6006329a80020418800ab
:101f0800105e88006349af002828ec006349ae00e2
:101f18002828ed0040418000610920000180e6008a
:101f28006349a900210320000100e6006349a800d5
:101f38008080eb0000f0a6008000eb0000020200a9
:101f4800000000000149880010498800615980009c
:101f5800705980000312240002002000560202007b
:101f680000000000fe0302000000000002a02000a4
:101f7800015020000180e6000200500080598800ce
:101f8800d15d8000e05d8000031224000200200083
:101f98005602020000000000fe03020000000000dc
:101fa80002a02000015020000180e600020050003d
:101fb800f05d8800f05d8000c34c80003200200096
:101fc8000218e700105e8000325e8000305e8800f4
:101fd80002005000800178000150200002a020007b
:101fe8000180e600820150008100ea000100e6005d
:101ff8008201400033548800c34388008059800020
:10200800f15d8000c34c8000320020000218e70018
:10201800115e80000218e7000000eb00010050008c
:10202800800178000150200002a020000180e60015
:10203800820150008100ea000100e60082014000b0
:10204800a4002000110009008401d8003041880054
:1020580003007800022820000298e60002007800b9
:102068000201ea000218e60002007800305a8800ef
:10207800b0438800305a8000011420000180e60037
:102088002a2aef000180e600100037008100ea00ec
:102098000100e6002a2aef000100e6000b003700e5
:1020a800305a8000515180000100400080017800c2
:1020b800429c20000298e600020078000201ea0033
:1020c8000218e6000200780050518800305a80005b
:1020d8008000eb0000f0a7008080eb000002020007
:1020e80000000000a33f240002002000be020200fe
:1020f8000000000093588000a25880005602020099
:1021080000000000b1548800c0548800305480009a
:102118008000eb0000f0a7008080eb0000020200c6
:1021280000000000831c240002002000be02020000
:1021380000000000b3588000c25880005602020018
:1021480000000000d1548800e054880050518000fd
:102158008000eb0000f0a7008080eb000002020086
:1021680000000000c361240002002400be02020037
:1021780000000000d3588000e25880005602020098
:1021880000000000f154880000558800b354800016
:10219800c25480004403020000000000d3548000b1
:1021a800e254800042030200000000006269af00b0
:1021b80001f0a200fe03020000000000a043880016
:1021c80000027800024b8000020040008001780085
:1021d800014b8000c10bb000024b8000c20bb10064
:1021e8000180e600810178000200e60082017800a3
:1021f800435188000400780000f0a7000000ea00be
:102208008000eb000002020000000000833424007c
:1022180002002000be0202000000000033598000c6
:1022280042598000560202000000000071558800e3
:1022380080558800b15d8000c05d80000349800042
:1022480002498000c44c8000350020000520e700ca
:1022580002003700e3488000f24880004203020091
:10226800000000006154880070548800fe030200da
:1022780000000000324b80000280e60004003700b6
:102288000201ea000280e600050037003900370045
:1022980091558000a05580006154880070548800d2
:1022a8002149800030498000831c2400020020005e
:1022b800be0202000000000013598000225980006d
:1022c8005602020000000000315588004055880081
:1022d8006154800070548000832424000200200090
:1022e800be02020000000000f3588000025980007e
:1022f8005602020000000000115588002055880091
:10230800335580004455800042030200000000005d
:1023180073558000825580004403020000000000cd
:102328006209af0001f0a200fe03020000000000f5
:10233800724b80000200400080017800714b8000e1
:10234800c10bb000724b8000c20bb1000180e600e7
:10235800810178000200e6008201780013518800ac
:10236800904b800020518800804b800030518800bd
:1023780000000600704b800010518800904a8000d1
:1023880020518800804b80003051880000000600f2
:1023980022212000904480000200e6009244880038
:1023a800704480000200e60072448800b044800057
:1023b8000200e600b2448800d04480000200e60033
:1023c800d2448800f2552000904480000280e60044
:1023d80092448800704480000280e60072448800bd
:1023e800b04480000280e600b2448800d0448000f7
:1023f8000280e600d24488003129af000700370088
:102408003ac9ae00050037003849af003ac9a900fb
:102418000000eb003849af00b0428800b0428000ad
:10242800310020000100e60004003700c0428000af
:10243800e10020000100e70000000600c04c800019
:10244800210020000180e600020037003049a90081
:102458003069a9000800fc00c04c80004100200041
:102468000180e6000700370000007800050033000f
:1024780000600100030037002b0037003a003700e6
:102488003900370062a9a9003849ae000d003700ad
:102498000f00fc00714a800041498800804a800092
:1024a8008100400051498800904a80008100400026
:1024b80061498800a04a8000810040007149880075
:1024c8000000060062a9a9003ac9af00420037001f
:1024d8000c48af00eeff37001400fc007144800088
:1024e800414988000001eb00904480000200e600aa
:1024f800804a80008100400051498800b044800033
:102508000200e600904a800081004000614988008e
:10251800d04480000200e600a04a8000810040000c
:1025280071498800000006003849ae00e5ff370011
:1025380062a9a8000f00fc001151800041498800e1
:1025480030518000810040005149880020518000ae
:1025580081004000614988004051800081004000ae
:1025680071498800000006003849af00c5ff3700f0
:102578003ac9af00180037001a00fc00115180005a
:102588003069ae0071448000414988000001eb00c9
:10259800904480000200e600804a800081004000ec
:1025a80051498800b04480000200e600904a80004b
:1025b8008100400061498800405180003049ae00e8
:1025c800d04480000200e600a04a8000810040005c
:1025d80071498800000006000f00fc0011458000ca
:1025e8004149880020458000810040005149880009
:1025f80030458000810040006149880040458000e6
:10260800810040007149880000000600604a80008f
:102618000000e00004003200915980003809a90048
:102628000008e6003809a800f04980000000e00032
:1026380004003200815880003829a9000008e6000b
:102648003829a800344a8000a50020000520b900d8
:10265800114880003889a9000008e6003889a800d8
:1026680021488000c01220000008e600040037005e
:102678004042200038a9a9000008e60038a9a800af
:102688004409e2000f003200244a8000431f200062
:102698000320b900f3598000025a800038c9a90004
:1026a8000198e60001003700060037000118e7002e
:1026b8000200370038c9a800020037000090e60081
:1026c80038c9a800104a8000017d20000102b90025
:1026d8008000eb004206200011000900422ad800c1
:1026e8005248800002034000104a80004106200042
:1026f8000102b90038e9a90004b0e60038e9a800e9
:102708003a09ae000000060040488000c1122000cf
:102718000180e6003aa9a9000c68af000e00370056
:1027280090598000a10020003a29af0061002000e4
:102738000100e6000000060030588000410120003a
:102748003a29af00110420000100e600000006004d
:102758000c68a8003aa9a9009059800051002000ef
:102768003a29af00310020000180e6000000060091
:1027780030588000410120003a29af0011042000a0
:102788000180e600000006003aa9a8000c68a9002c
:10279800000006003849af002028ef002028ec0090
:1027a80001418000900020000008e6004400370046
:1027b800a000200000418800c04c800021002000bb
:1027c8000180e7002a2aef0060448000c10d200044
:1027d8000180e6003a00370050458000c10d200016
:1027e8000180e600360037005045800001052000d2
:1027f8000100e6003200370060448000910b2000a1
:102808000100e600750037005e08e20006003a00a5
:1028180050458000910b20000180e6002a00370017
:102828005e28ec00280037005c28ef005e28ec00ea
:10283800f0428000510020000100e600220037002d
:102848005628ec00c04c8000110020000180e600f2
:1028580006003a003ac9a900b042800041002000b1
:102868000180e6005628ef0015003700b0428000ce
:10287800510020000180e6005628ef003ac9a9005f
:10288800410020000100e7003ac9a8000100e70064
:102898003129a900410020000180e7000800370025
:1028a80070448000104588009044800020458800ce
:1028b800b044800030458800d044800040458800fe
:1028c8005c28ef005e28ef006044800050458800d7
:1028d8003ac9ae00000006003849af000000060003
:1028e8003109a80010458000e003b0007144800061
:1028f8000088e6001500370010458000e003b100ad
:10290800714480000008e600190037004045800047
:10291800e003b000d14480000088e6001d003700c5
:1029280040458000e003b100d14480000008e60083
:10293800210037004e28ef005028ef005228ef0002
:102948005428ef003109a900000006004e28ec00c9
:1029580070428000e10120000180e600800037001d
:102968005028ef005228ef005428ef00000006001e
:102978005028ec0080428000e10120000180e60040
:10298800930037004e28ef005228ef005428ef003c
:10299800000006005228ec0090428000e10120006f
:1029a8000180e6007d0337004e28ef005028ef0035
:1029b8005428ef00000006005428ec00a0428000d4
:1029c800e10120000180e600150337004e28ef00e2
:1029d8005028ef005228ef00000006005e28ef00a4
:1029e8003ac9af00b6ff3700604480007108200084
:1029f8000180e600b2ff37005c08e20006003a00fa
:102a080050458000710820000100e600acff370047
:102a18005c28ec00acff370060448000a105200072
:102a28000100e600a6ff37005c28ec00e0428000c9
:102a3800f10020000100e600a3ff3700362aec0071
:102a4800b0518000310020000180e600362aef00f6
:102a58002a2aef00004b8000405188003049a90025
:102a68003069a900b0518000110020000100e70082
:102a78003049a800210020000100e7003069a800c3
:102a88003089ae003049a90030a9ae003069a900ec
:102a9800c04c8000210020000180e60088ff37003c
:102aa8003049a9003069a90085ff370040438000fc
:102ab800314380000008e700000006003a69a900d9
:102ac8006808e2005c003a003043800041092000b9
:102ad8000180e7000d0037003ac9af003ac9a900e4
:102ae8003009a9003029a900382aef003a2aef0056
:102af8003c2aef005628ec00b0428000510020002c
:102b08000100e7005628ef004b003700b042800074
:102b1800e400680048003a003043800001092000c2
:102b28000180e700170037003009a9003ac9af0053
:102b38000b003700380ae20043003a003a0ae20084
:102b480025013a003c0ae20094013a005828ed00b9
:102b580039003b00d0012000c04288003600370011
:102b68005028ef004e28ef005228ef005428ef00bd
:102b78005a28ed0030003b0020012000d042880098
:102b88002d00370030438000110920000180e70044
:102b9800190037003009a9003ac9af000c00370006
:102ba800380ae2009a003a003a0ae200f7013a00cd
:102bb8003c0ae20043023a005828ec00c042800078
:102bc800e10120000100e7005828ef001a00370053
:102bd8005028ef004e28ef005228ef005428ef004d
:102be8005a28ec00d0428000310120000180e60024
:102bf8005a28ef00100037003043800021092000d8
:102c08000180e700040037003ac9af0084023700aa
:102c1800dd04370008003700304380003109200008
:102c28000180e700040037003ac9af00db02370033
:102c380030053700000037003109a9003043800013
:102c48004043880000000600c051800011002000a9
:102c58000180e7000f0037008229ec00104c80004b
:102c6800c1052000020320000180e600124c880004
:102c7800110420000180e600efff370091032000d7
:102c88000100e600ecff370012042000124c880017
:102c9800e9ff3700210020000180e7000f0037001e
:102ca8008429ec00204c8000c1052000020320008c
:102cb8000180e600224c8800110420000180e60013
:102cc800ddff3700910320000100e600daff37003e
:102cd80012042000224c8800d7ff37003100200062
:102ce8000180e7000f0037008629ec00304c800097
:102cf800c1052000020320000180e600324c880054
:102d0800110420000180e600cbff3700910320006a
:102d18000100e600c8ff370012042000324c88008a
:102d2800c5ff3700410020000180e7000f00370091
:102d38008829ec00404c8000c105200002032000d7
:102d48000180e600424c8800110420000180e60062
:102d5800b9ff3700910320000100e600b6ff3700f5
:102d680012042000424c8800b3ff370051002000b5
:102d78000180e7000f0037008a29ec00504c8000e2
:102d8800c1052000020320000180e600524c8800a3
:102d9800110420000180e600a7ff370091032000fe
:102da8000100e600a4ff370012042000524c8800fe
:102db800a1ff3700610020000180e7000f00370005
:102dc8008c29ec00604c8000c10520000203200023
:102dd8000180e600624c8800110420000180e600b2
:102de80095ff3700910320000100e60092ff3700ad
:102df80012042000624c88008fff37007100200009
:102e08000180e7008cff370062c9aa008aff3700fb
:102e1800c0518000110020000180e7000f0037003a
:102e28008229ed00104c8000f1022000b20520003c
:102e38000100e600124c8800910320000100e60022
:102e48007dff3700110420000180e6007aff37007b
:102e580092032000124c880077ff370021002000e1
:102e68000180e7000f0037008429ed00204c800026
:102e7800f1022000b20520000100e600224c880083
:102e8800910320000100e6006bff370011042000c9
:102e98000180e60068ff370092032000224c88007a
:102ea80065ff3700310020000180e7000f00370080
:102eb8008629ed00304c8000f1022000b205200088
:102ec8000100e600324c8800910320000100e60072
:102ed80059ff3700110420000180e60056ff370033
:102ee80092032000324c880053ff37004100200035
:102ef8000180e7000f0037008829ed00404c800072
:102f0800f1022000b20520000100e600424c8800d2
:102f1800910320000100e60047ff3700110420005c
:102f28000180e60044ff370092032000424c8800ed
:102f380041ff3700510020000180e7000f003700f3
:102f48008a29ed00504c8000f1022000b2052000d3
:102f58000100e600524c8800910320000100e600c1
:102f680035ff3700110420000180e60032ff3700ea
:102f780092032000524c88002fff37006100200088
:102f88000180e7000f0037008c29ed00604c8000bd
:102f9800f1022000b20520000100e600624c880022
:102fa800910320000100e60023ff370011042000f0
:102fb8000180e60020ff370092032000624c880061
:102fc8001dff3700710020000180e7001aff37005d
:102fd80062c9aa0018ff3700d051800011002000f4
:102fe8000180e700060037004c2aec00a100200011
:102ff800605280000180e6004c2aef004b00370049
:10300800d0518000210020000180e7000600370031
:103018004e2aec00a1002000705280000180e600da
:103028004e2aef0041003700d051800031002000c7
:103038000180e70006003700502aec00a1002000bc
:10304800805280000180e600502aef0037003700e8
:10305800d0518000410020000180e70006003700c1
:10306800522aec00a1002000905280000180e60066
:10307800522aef002d003700d05180005100200067
:103088000180e70006003700542aec00a100200068
:10309800a05280000180e600542aef002300370088
:1030a800d0518000610020000180e7000600370051
:1030b800562aec00a1002000b05280000180e600f2
:1030c800562aef0019003700d05180007100200007
:1030d8000180e70006003700582aec00a100200014
:1030e800c05280000180e600582aef000f00370028
:1030f800d0518000810020000180e70006003700e1
:103108005a2aec00a1002000d05280000180e6007d
:103118005a2aef0005003700d051800091002000a6
:103128000180e700c4fe37005e0aaa00f052800062
:10313800905f8800c0a4200041bf2000b01878002c
:10314800b0187800b0187800b0187800b018780077
:10315800b0187800b0187800b01878007000200017
:10316800be0e020000000000415f8000914c880004
:10317800305f8000804c88000002020000000000e0
:10318800a3c52400920e2900be0202000000000020
:103198003152880020528800a7fe3700e051800095
:1031a800110020000180e70006003700602aec00cb
:1031b80021002000005380000180e600602aef0013
:1031c80055003700e0518000210020000180e70011
:1031d80006003700622aec00a1002000105380008e
:1031e8000180e600622aef004b003700e0518000c2
:1031f800310020000180e70006003700642aec0057
:10320800a1002000205380000180e600642aef001e
:1032180041003700e0518000410020000180e700b4
:1032280006003700662aec00a10020003053800019
:103238000180e600662aef0037003700e051800081
:10324800510020000180e70006003700682aec00e2
:10325800a1002000405380000180e600682aef00aa
:103268002d003700e0518000610020000180e70058
:10327800060037006a2aec00a100200050538000a5
:103288000180e6006a2aef0023003700e051800041
:10329800710020000180e700060037006c2aec006e
:1032a800a1002000605380000180e6006c2aef0036
:1032b80019003700e0518000810020000180e700fc
:1032c800060037006e2aec00a10020007053800031
:1032d8000180e6006e2aef000f003700e051800001
:1032e800910020000180e70006003700702aec00fa
:1032f800a1002000805380000180e600702aef00c2
:1033080005003700e0518000a10020000180e7009f
:1033180049fe3700720aaa0090538000905f880027
:1033280000a6200041bf2000b0187800b01878002f
:10333800b0187800b0187800b0187800b018780085
:10334800b0187800b0187800b01878008000200015
:10335800be0e020000000000415f8000b14c8800f2
:10336800305f8000a04c88000002020000000000ce
:10337800a3c52400920e2900be020200000000002e
:1033880051528800405288002bfe3700d0518000ef
:10339800110020000180e700050037004c2aed00ed
:1033a80062ff3b0093002000635288005fff3700f4
:1033b800d0518000210020000180e700050037007f
:1033c8004e2aed0059ff3b009300200073528800fd
:1033d80056ff3700d0518000310020000180e700ff
:1033e80005003700502aed0050ff3b0093002000f5
:1033f800835288004dff3700d051800041002000e3
:103408000180e70005003700522aed0047ff3b0026
:10341800930020009352880044ff3700d051800069
:10342800510020000180e70005003700542aed0014
:103438003eff3b0093002000a35288003bff37006b
:10344800d0518000610020000180e70005003700ae
:10345800562aed0035ff3b0093002000b352880048
:1034680032ff3700d0518000710020000180e70052
:1034780005003700582aed002cff3b009300200080
:10348800c352880029ff3700d051800081002000f6
:103498000180e700050037005a2aed0023ff3b00b2
:1034a80093002000d352880020ff3700d0518000bd
:1034b800910020000180e700dffd37005e0aaa00c6
:1034c8001aff3700e0518000110020000180e7005a
:1034d80005003700602aed008fff3b001300200035
:1034e800035388008cff3700e05180002100200042
:1034f8000180e70005003700622aed0086ff3b00e7
:10350800930020001353880083ff3700e0518000a8
:10351800310020000180e70005003700642aed0033
:103528007dff3b0093002000235388007aff37007b
:10353800e0518000410020000180e70005003700cd
:10354800662aed0074ff3b00930020003353880087
:1035580071ff3700e0518000510020000180e70032
:1035680005003700682aed006bff3b009300200040
:103578004353880068ff3700e05180006100200055
:103588000180e700050037006a2aed0062ff3b0072
:1035980093002000535388005fff3700e0518000fc
:1035a800710020000180e700050037006c2aed005b
:1035b80059ff3b00930020006353880056ff3700f3
:1035c800e0518000810020000180e70005003700fd
:1035d8006e2aed0050ff3b009300200073538800d3
:1035e8004dff3700e0518000910020000180e70086
:1035f80005003700702aed0047ff3b0093002000cc
:103608008353880044ff3700e0518000a100200068
:103618000180e70088fd3700720aaa003eff3700e4
:103628005028ef004e28ef005228ef005428ef00f2
:10363800d04280000000e000b7003200d042800095
:10364800e1006800ba003200d0428000e200680061
:10365800c3003200d0428000e3006800cc00320092
:10366800d0428000e4006800d5003200d0428000db
:10367800e5006800f6003200d0428000e6006800ed
:10368800f5003200d0428000e700680002013200f5
:10369800d0428000e80068000b013200d042800070
:1036a800e900680014013200d0428000ea00680096
:1036b8001d013200d0428000eb0068002601320074
:1036c800d0428000ec00680037013200d042800010
:1036d800ed006800ef013200d0428000ee00680083
:1036e800fe013200d0428000ef0068000d02320077
:1036f800d0428000f00068000f023200d042800003
:10370800f100680011023200d0428000f200680027
:1037180089013200d0428000f30068008b0132003a
:10372800d0428000f40068008a013200d042800054
:10373800f500680089013200d0428000f600680078
:1037480088013200d0428000f7006800870132000b
:10375800d0428000f800680086013200d042800024
:10376800f90068008e013200d0428000fa0068003b
:103778009c013200d0428000fb006800a4013200a6
:10378800d0428000fc006800ac013200d0428000ca
:10379800fd006800af01320027fd37005028ef0018
:1037a8004e28ef005228ef005428ef00d042800046
:1037b8000000e000ff003200d0428000e100680015
:1037c80001013200d0428000e200680009013200a5
:1037d800d0428000e300680011013200d04280002e
:1037e800e400680076003200d0428000e5006800fe
:1037f80097003200d0428000e600680013013200d2
:10380800d0428000e70068001f013200d0428000eb
:10381800e800680027013200d0428000e900680013
:103828002f013200d0428000ea00680037013200e0
:10383800d0428000eb006800c7003200d042800010
:10384800ec006800d8003200d0428000ed0068002b
:1038580090013200d0428000ee0068009f013200e3
:10386800d0428000ef006800ae013200d0428000f4
:10387800f0006800b0013200d0428000f10068001a
:10388800ba013200d0428000f20068002a013200fa
:10389800d0428000f30068002c013200d042800042
:1038a800f40068002b013200d0428000f500680067
:1038b8002a013200d0428000f60068002901320057
:1038c800d0428000f700680028013200d042800012
:1038d800f80068002d013200d0428000f90068002d
:1038e8002f013200d0428000fa0068004301320004
:1038f800d0428000fb0068004b013200d0428000bb
:10390800fc00680059013200d0428000fd006800c8
:103918005b013200c8fc37005829ec00710920000f
:10392800c04a80000180e6005829ef00c2fc370039
:103938005a29ec0071092000d04a80000180e60075
:103948005a29ef008000eb00d04a800000020200f4
:103958000000000091588800a0588800b6fc370085
:103968005c29ec0071092000e04a80000180e60033
:103978005c29ef008000eb00e04a800000020200b2
:1039880000000000b1588800c0588800aafc370021
:103998005e29ec0071092000f04a80000180e600f1
:1039a8005e29ef008000eb00f04a80000002020070
:1039b80000000000d1588800e05888009efc3700bd
:1039c80090418000004d88004828ae000200370072
:1039d800b0418000204d8800204d8000014d8000be
:1039e800010050008000eb0000020200000000000f
:1039f8000348240002002000be020200000000006c
:103a08006148880070488800d04480003109af00c0
:103a180040458000004b8800222120000200e6007b
:103a2800024b8800f25520000280e600024b880015
:103a3800004b8000030120000300b900430620006a
:103a4800110009004308d800b05588007afc3700f7
:103a58006269aa0078fc37006429ec00910c200008
:103a6800204b80000180e6006429ef008000eb0015
:103a7800204b800000020200000000000312240016
:103a8800020020005602020000000000b15d88001c
:103a9800c05d880068fc37006629ec00910c2000a6
:103aa800304b80000180e6006629ef008000eb00c3
:103ab800304b800000020200000000009155880091
:103ac800a05588005cfc37006829ec0071092000cb
:103ad800404b80000180e6006829ef008000eb0081
:103ae800404b80000002020000000000f1588800ee
:103af8000059880050fc37006a29ec007109200041
:103b0800504b80000180e6006a29ef008000eb003e
:103b1800504b80000002020000000000115988008c
:103b28002059880044fc37006c29ec0071092000fa
:103b3800604b80000180e6006c29ef008000eb00fc
:103b4800604b80000002020000000000315988002c
:103b58004059880038fc370070418000f04c8800dc
:103b6800704480003109af0010458000704b880018
:103b7800222120000200e600724b8800f255200046
:103b88000280e600724b8800704b80000301200021
:103b98000300b90043062000110009004308d800bb
:103ba800c055880024fc37006209aa004808a9000b
:103bb80021fc37005829ed0002003b006309200072
:103bc800c34a88001cfc37005a29ed0002003b005c
:103bd80063092000d34a88008000eb00d04a8000a7
:103be800000202000000000091588800a0588800d8
:103bf80011fc37005c29ed0002003b00630920003e
:103c0800e34a88008000eb00e04a800000020200de
:103c180000000000b1588800c058880006fc370032
:103c28005e29ed0002003b0063092000f34a88008a
:103c38008000eb00f04a8000000202000000000053
:103c4800d1588800e0588800fbfb37006429ed0054
:103c580002003b00830c2000234b88008000eb000f
:103c6800204b800000020200000000000312240024
:103c7800020020005602020000000000b15d88002a
:103c8800c05d8800ecfb37006629ed0002003b00b0
:103c9800830c2000334b88008000eb00304b800001
:103ca800000202000000000091558800a05588001d
:103cb800e1fb37006829ed0002003b0063092000a2
:103cc800434b88008000eb00404b8000000202005c
:103cd80000000000f158880000598800d6fb370022
:103ce8006a29ed0002003b0063092000534b88005d
:103cf8008000eb00504b8000000202000000000032
:103d08001159880020598800cbfb37006c29ed0039
:103d180002003b0063092000634b88008000eb0031
:103d2800604b80000002020000000000315988004a
:103d380040598800c0fb37003109af00befb37008f
:103d48003129a9003ac9a900bbfb37007689aa0026
:103d5800b9fb37007669aa00b7fb37007609aa00d5
:103d6800b5fb37007629aa00b3fb37007649aa00cd
:103d7800b1fb37007829ec0031032000c04b8000ec
:103d88000180e6007829ef00abfb37007829ed00c9
:103d980002003b0023032000c34b8800a6fb37002a
:103da80070418000204d8800b0418000104d88008f
:103db800204d8000014d8000010050008000eb0084
:103dc8000002020000000000034824000200200056
:103dd800be020200000000006148880070488800a8
:103de80095fb37004c28ec0011052000604280004c
:103df8000180e6004c28ef008ffb37004c28ed00cf
:103e080002003b0003052000634288008afb37005c
:103e18004a28ec0011052000504280000180e6008d
:103e28004a28ef0084fb37004a28ed0002003b00d7
:103e380003052000534288007ffb37009a29ec00d5
:103e480031002000d04c80000180e6009a29ef0064
:103e580079fb37009c29ec0031002000e04c800001
:103e68000180e6009c29ef0073fb37009a29ed00da
:103e780002003b0023002000d34c88006efb370073
:103e88009c29ed0002003b0023002000e34c880041
:103e980069fb3700b04480003109af00304580002d
:103ea800904b8800222120000200e600924b8800f7
:103eb800f25520000280e600924b8800904b80006b
:103ec800030120000300b900430620001100090087
:103ed8004308d800d055880057fb3700904480002d
:103ee8003109af0020458000804b88002221200046
:103ef8000200e600824b8800f25520000280e600ae
:103f0800824b8800804b8000030120000300b90029
:103f180043062000110009004308d800e055880036
:103f280045fb37003089aa0062e9a9003089af0053
:103f380062e9a80040fb370030a9aa006309a9007c
:103f480030a9af006309a8003bfb37003109af0077
:103f580039fb37009829ec00c04c80004100200054
:103f68000180e6009829ef0033fb37003109af00e4
:103f780031fb37009829ed002ffb3b003000200073
:103f8800c04c88002cfb3700c04280000000e000d5
:103f9800bf013200c0428000e1006800b300320077
:103fa800c0428000e2006800bb003200c0428000ce
:103fb800e3006800c3003200c0428000e4006800eb
:103fc800c1003200c0428000e5006800c90032002c
:103fd800c0428000e6006800d1003200c042800084
:103fe800e7006800d9003200c0428000e80068009d
:103ff800e4003200c0428000e9006800ec003200b2
:10400800c0428000ea00680057013200c0428000c8
:10401800eb00680056013200c0428000ec006800e6
:1040280065013200c0428000ed0068006e01320078
:10403800c0428000ee0068008c013200c04280005f
:10404800ef00680086003200c0428000f00068007f
:1040580049013200c0428000f1006800e2003200ed
:10406800c0428000f2006800ef003200c0428000c9
:10407800f3006800fc003200c0428000f4006800d1
:1040880009013200c0428000f50068006101320079
:10409800c0428000f600680064013200c04280001f
:1040a800f700680018013200c0428000f80068007c
:1040b80017013200c0428000f90068001601320082
:1040c800c0428000fa00680015013200c04280003a
:1040d800fb00680018013200c0428000fc00680044
:1040e80017013200c0428000fd0068001a0132004a
:1040f800d1fa3700c04280000000e00064013200bd
:10410800c0428000e10068005e003200c0428000ca
:10411800e200680066003200c0428000e3006800e8
:1041280068003200c0428000e40068006c00320081
:10413800c0428000e500680074003200c042800080
:10414800e60068007c003200c0428000e70068009a
:1041580085003200c0428000e80068008f0032000d
:10416800c0428000e900680098003200c042800028
:10417800ea006800fc003200c0428000eb006800e2
:10418800fb003200c0428000ec00680011013200e0
:10419800c0428000ed00680019013200c042800072
:1041a800ee00680031013200c0428000ef00680074
:1041b8002b003200c0428000f0006800ee003200a0
:1041c800c0428000f100680087003200c0428000d1
:1041d800f200680094003200c0428000f3006800da
:1041e800a1003200c0428000f4006800ae00320036
:1041f800c0428000f500680012013200c042800011
:10420800f600680014013200c0428000f700680020
:10421800bd003200c0428000f8006800bc003200d7
:10422800c0428000f9006800bb003200c042800034
:10423800fa006800ba003200c0428000fb00680043
:10424800bd003200c0428000fc006800bc003200a3
:10425800c0428000fd006800bf00320076fa3700d7
:104268003a29aa003aa9a90073fa37003c29ec00b8
:1042780051062000e04980000180e6003c29ef005b
:104288006dfa37003c29ed006bfa3b00430620002d
:10429800e349880068fa37003e29ec00e102200073
:1042a800f04980000180e6003e29ef0062fa3700fd
:1042b8003e29ed0060fa3b00d3022000f349880054
:1042c8005dfa37000000fe004029ec005100200094
:1042d800004a80000180e6004029ef0056fa3700c6
:1042e8004029ed0054fa3b0043002000034a8800af
:1042f80051fa37004229ec0051062000104a80008c
:104308000180e6004229ef004bfa37004229ed0010
:1043180049fa3b0043062000134a880046fa370052
:104328004429ec0051062000204a80000180e60064
:104338004429ef0040fa37004429ed003efa3b00db
:1043480043062000234a88003bfa37004629ec0040
:10435800b10f2000304a8000c30320000180e6002e
:10436800334a880034fa37004629ed00b1032000ab
:10437800304a8000a30f20000100e600334a88007d
:104388002dfa37004829ec0051062000404a8000e9
:104398000180e6004829ef0027fa37004829ed0098
:1043a80025fa3b0043062000434a880022fa3700da
:1043b8004aa9ec00f1152000504a8000a30520000e
:1043c8000180e600534a88001bfa37004aa9ed002d
:1043d80091052000504a8000e31520000100e60006
:1043e800534a880014fa370070448000704a8800e5
:1043f800222120000200e600724a8800f2552000bf
:104408000280e600724a8800704a8000030120009a
:104418000300b90043062000110009004308d80032
:10442800f055880004fa370090448000804a8800dc
:10443800222120000200e600824a8800f25520006e
:104448000280e600824a8800804a8000030120003a
:104458000300b90043062000110009004308d800f2
:1044680000568800f4f93700b0448000904a88006c
:10447800222120000200e600924a8800f25520001e
:104488000280e600924a8800904a800003012000da
:104498000300b90043062000110009004308d800b2
:1044a80010568800e4f93700d0448000a04a8800fc
:1044b800222120000200e600a24a8800f2552000ce
:1044c8000280e600a24a8800a04a8000030120007a
:1044d8000300b90043062000110009004308d80072
:1044e80020568800d4f9370080568000d04b8800c9
:1044f80090568000e04b8800cff93700a056800026
:10450800f04b8800ccf9370056a9aa00caf9370041
:104518005669aa00c8f937005649aa00c6f93700f3
:104528005689aa00000820005689ae000000200025
:10453800f0518800c0f937008e29aa00bef937006b
:104548008e09aa00000820005689ae00000020004d
:10455800f0518800b8f937003a69a80048400200cd
:1045680000000000b4f937003a89aa00b2f9370010
:104578005629aa00b0f937006289aa009829ef00e5
:104588006289ae003049a9006289ae003069a9008d
:104598006289ae00040037000400fc00e0932400a8
:1045a80040098800a4f937000400fc00f0ff270048
:1045b80040098800a0f937003009a8007429ec00e8
:1045c800f1012000a04b80000180e6007429ed0075
:1045d80099f937003009a8007429ed0096f93b00d5
:1045e8007429ec0094f93700382aec008100200087
:1045f800c05180000180e600382aef008ef93700ac
:10460800382aed008cf93b0073002000c351880064
:1046180089f937003a2aec00a1002000d051800027
:104628000180e6003a2aef0083f937003c2aec00c3
:10463800b1002000e05180000180e6003c2aef0034
:104648007df937003a2aed007bf93b009300200002
:10465800d351880078f937003c2aed0076f93b0001
:10466800a3002000e351880073f93700b0448000ac
:10467800004c8800030120000300b9004306200015
:10468800110009004308d800305688006af937003d
:104698003129a8003ac9a800704480001045880054
:1046a8009044800020458800b04480003045880050
:1046b800d0448000404588005ff9370000000600bc
:1046c80060438000011020000100e6001c00370054
:1046d8008000eb006de8af008080eb006043800055
:1046e800000202000000000043da2300f2ff2f005e
:1046f80056020200000000003a29ae00040037000c
:10470800fe0302000000000050438800000006007d
:1047180003202400020020004203020000000000e1
:10472800e3f02300428e230056020200000000003e
:10473800fe0302000000000050438800000006004d
:104748008000eb0071e8af008080eb0080438000c0
:10475800000202000000000043da2300f2ff2f00ed
:1047680056020200000000003a29af00040037009a
:10477800fe0302000000000050438800000006000d
:1047880063fe230062662600560202000000000055
:10479800fe030200000000000202200002004000a8
:1047a80050438800000006000002020000000000dc
:1047b80073f22300f24723005602020000000000b3
:1047c800fe0302000000000000000600f401fc00e7
:1047d8000002020000000000834880009248800028
:1047e80042030200000000004009e2000a00320013
:1047f800054a800061836a000a00320062836a0009
:104808000b00320063836a000c003200931424000a
:1048180012f629000c0037009304240012f6290030
:1048280009003700930c240012f62900060037000f
:104838006310240012a4260003003700731124001b
:10484800f28829000000370056020200000000002c
:1048580001f0a600020037008000eb000000eb002a
:10486800a1488800b0488800fe030200000000004c
:104878004048880001f0a7000829ef000100e00087
:104888000100320000000600120020000200e600cd
:1048980000000600a1488000b0488000937e2300f5
:1048a80042452000560202000000000001f0a70067
:1048b80006003700c3488000d24880004403020045
:1048c80000000000c1488800d0488800fe030200ac
:1048d8000000000001f0a600504888000000060013
:1048e800c0418000a1418000aa240200000000000d
:1048f800a0418000d1418000d0418800c02402003e
:1049080000000000d6240200000000000425020078
:1049180000000000e041800081418000aa240200dc
:104928000000000080418000f1418000f0418800d3
:10493800c0240200000000009625020000000000cc
:10494800c42502000000000000000600010050001d
:104958008001780001802000020021000180e6002b
:10496800820150008100ea000100e6008201400057
:104978000342880000000600010050008001780012
:1049880001802000020021000180e6008201500021
:104998008100ea000100e60082014000134288001d
:1049a8000000060000428000012020000180e6008f
:1049b8004428ef000180e600100037008100ea007b
:1049c8000100e6004428ef000100e6000b00370074
:1049d80000428000214280000100400080017800f0
:1049e800025327000298e600020078000201ea005c
:1049f8000218e60002007800204288000000060045
:104a0800004280008000eb0000f0a7008080eb00ef
:104a18000002020000000000a33f24000200200062
:104a2800be0202000000000093588000a2588000d7
:104a38005602020000000000b1548800c0548800eb
:104a4800104280008000eb0000f0a7008080eb009f
:104a58000002020000000000831c24000200200065
:104a6800be02020000000000b3588000c258800057
:104a78005602020000000000d1548800e05488006b
:104a8800204280008000eb0000f0a7008080eb004f
:104a98000002020000000000c3612400020024009c
:104aa800be02020000000000d3588000e2588000d7
:104ab8005602020000000000f154880000558800ea
:104ac800b3548000c2548000440302000000000078
:104ad800d3548000e254800042030200000000002a
:104ae8006269af0001f0a200fe03020000000000ae
:104af800024b80000200400080017800014b8000da
:104b0800c10bb000024b8000c20bb1000180e6006f
:104b1800810178000200e600820178004351880094
:104b28000000060000428000012020000180e6000d
:104b38004628ef000180e600100037008100ea00f7
:104b48000100e6004628ef000100e6000b003700f0
:104b5800004280003142800001004000800178005e
:104b6800025327000298e600020078000201ea00da
:104b78000218e600020078003042880000000600b3
:104b8800004280008000eb0000f0a7008080eb006e
:104b98000002020000000000a33f240002002000e1
:104ba800be02020000000000f35880000259800095
:104bb80056020200000000001155880020558800a8
:104bc800104280008000eb0000f0a7008080eb001e
:104bd8000002020000000000831c240002002000e4
:104be800be02020000000000135980002259800014
:104bf8005602020000000000315588004055880028
:104c0800304280008000eb0000f0a7008080eb00bd
:104c18000002020000000000c3612400020024001a
:104c2800be020200000000003359800032598000a3
:104c380056020200000000005155880060558800a7
:104c48001355800022558000440302000000000034
:104c580033558000425580004203020000000000e6
:104c68006209af0001f0a200fe030200000000008c
:104c7800724b80000200400080017800714b800078
:104c8800c10bb000724b8000c20bb1000180e6007e
:104c9800810178000200e600820178001351880043
:104ca8000000060070418000f14c800001005000b7
:104cb8008000eb0000f0a7008080eb0000020200fb
:104cc800000000006348800072488000be020200b5
:104cd80000000000fe030200000000008041880080
:104ce800014020000180e6008141880001c02f00ba
:104cf8000100e60081418800b0418000114d80002c
:104d08000100500006003b00804180000180200027
:104d180000f0a70001802f0000805000804188002b
:104d280090418000014d8000010050008000eb00a0
:104d380000f0a7008080eb000002020000000000e5
:104d48006348800072488000be0202000000000034
:104d5800fe03020000000000a0418800014020007e
:104d68000180e600a141880001c02f000100e60093
:104d7800a1418800b0418000114d80000100500021
:104d880006003b00a04180000180200000f0a70041
:104d980001802f0000805000a0418800000006001c
:104da8008000eb0007ebaf008080eb0030588000fc
:104db8000002020000000000810178000001780074
:104dc8005602020000000000d15c8800e05c880008
:104dd800d1598000e0598000000202000000000064
:104de80081017800000178005602020000000000ee
:104df800d35c8000e25c80004403020000000000f5
:104e08007a04020000000000fe0302000000000017
:104e1800f1598800005a880000000600d159800026
:104e2800e05980000002020000000000d15c880008
:104e3800e05c88008000eb0007ebaf008080eb00af
:104e4800305880000002020000000000d35c80009f
:104e5800e25c8000400402000000000053262400a9
:104e680012ee22005602020000000000fe030200bb
:104e78000000000080588800000006000ac8a90049
:104e88000ae8a9000b88a900e6cd20000b68af004e
:104e9800e6de2000b6027800770420000728e70045
:104ea80026003700670520000728e70004003700c0
:104eb800270520000728e7004f0037008b0437003c
:104ec800b60278004705200007a8e70000000600a2
:104ed800b60278007704200007a8e7000000060063
:104ee80086cd20000b68af0086de200098002000e9
:104ef8006700070029c82000980020006b00070001
:104f080048002000620007009800200060000700a9
:104f1800480020005e000700880020005c000700b1
:104f2800480020005a00070009c920008800200016
:104f38005e0007000ae8a80000000600b602780034
:104f48007704200007a8e70000000600b6027800f2
:104f58001704200007a8e7000000060086cd2000ff
:104f68000b68af0086de200098002000480007008c
:104f7800d80020004600070049c12000e8002000b2
:104f88004a000700c9c22000480020004700070067
:104f980009c32000f800200044000700a9c420002d
:104fa8004800200041000700e9c420004800200014
:104fb8003e00070029c52000580020003b000700dc
:104fc80089c52000680020003800070029c6200095
:104fd800980020003500070029c72000980020000d
:104fe800320007000ac8a8000a28ae000000060020
:104ff8000a28a90000000600b6027800d70420009d
:1050080007a8e70000000600b60278003704200071
:1050180007a8e7000000060086cd20000b68af0057
:1050280086de20009800200019000700d800200024
:105038001700070089cc2000480020001b0007004b
:10504800b8002000120007004800200010000700e8
:10505800c80020000e000700480020000c000700d0
:10506800980020000a000700a80020000800070098
:10507800a9cc2000880020000c0007000b88a8009d
:105088000a28ae00000006000a28a9000000060051
:105098000804e90015043200b6027800c7022000af
:1050a80007a8e700faff3700000006000804e90037
:1050b8000e043200b6027800851c7800c702200072
:1050c80007a8e700f9ff37000000060069f30700aa
:1050d800a6cc200049bf2000a0cd20005060880049
:1050e800f8280200000000000ba8af00000006002e
:1050f800405f800060578800305f800070578800ec
:10510800000006005bf3070086c5200049bf2000a9
:1051180060c62000506088009e2802000000000041
:10512800305f800080578800a05780009057880023
:10513800000006000bc8a900f42aef000004eb00e9
:10514800082cef00f20ba900082cec008002eb0001
:10515800b6027800c70220000728e70015003700cc
:10516800e70220000728e7000f003700576080009b
:105178000638e60018003700d70220000728e700a5
:1051880006003700f700200087836200871c78003c
:105198000bc8af000804e800ebff3700f20ba800cb
:1051a800082ced00e8ff37000bc8a800082ced001c
:1051b800e5ff3700082ced00a8578800080ce2002e
:1051c80005003200080ced00be0e020000000000d1
:1051d8000ba8a90000000600e62bef00e82bef0063
:1051e8000ba8a80000000600082cef00f20ba9008d
:1051f800082cec00b6027800c70220000728e70058
:1052080010003700e70220000728e7000d003700ec
:10521800576080000638e60012003700d7022000e9
:105228000728e70004003700f700200087836200a2
:10523800871c7800eeff3700f20ba800082ced0061
:10524800ebff3700082ced00080ce20005003200e7
:10525800080ced00be0e0200000000000ba8a9001b
:1052680000000600e62bef00e82bef000ba8a800d3
:1052780000000600fff2070026c5200049bf2000f5
:1052880080c5200050608800082cef00082cec0036
:10529800b6027800f700200087836200871c780038
:1052a800c70220000728e700040037005760800085
:1052b8000638e60001003700f4ff37008024eb00d1
:1052c800082ced0000003700080ce20087033200cc
:1052d800080ced00be0e020000000000305f8000e8
:1052e800a05988003e0f020000000000766280008e
:1052f800f500200005036300a65f88000000200079
:10530800be0e020000000000305f8000b059880027
:1053180000000600d7f2070006c9200049bf200098
:1053280020ca2000506088009e280200000000006b
:10533800415f8000305f80003a29af0017003700d6
:10534800a55780000500e0001200320061836a0062
:105358000d00320062836a000700320063836a002e
:10536800010032002a003700833e200011000900a6
:105378004308d80007003700430620001100090041
:105388004308d80003003700a300200011000900db
:105398004308d80090598800000006000002020067
:1053a80000000000a55780000500e0001000320052
:1053b80061836a000b00320062836a0006003200d3
:1053c80063836a000100320011003700834c240017
:1053d80002002000080037000332240002002000e9
:1053e80005003700031824000200200002003700df
:1053f800c3fc2300d2cc2c00be0202000000000037
:10540800fe0302000000000090598800000006001a
:10541800322bef000000060096f2070026c8200095
:1054280049bf200040c92000506088009e28020023
:1054380000000000415f8000305f80000002020031
:1054480000000000a55780000500e0000f003200b2
:1054580061836a000b00320062836a000600320032
:1054680063836a00010032006c003700a347240000
:105478000200200005003700832c240002002000d1
:10548800020037000312240002002000be020200be
:1054980000000000d15d8800e05d8800fe03020086
:1054a8000000000000588800d15d8000e05d8000a9
:1054b80063f3230012b62000560202000000000029
:1054c800d15d8800e05d8800fe0302000000000056
:1054d800f05788000000060066f2070026c7200083
:1054e80049bf200040c82000506088009e28020064
:1054f80000000000415f8000305f8000e04d8800c0
:10550800000006005bf2070026c6200049bf200005
:1055180040c72000506088009e280200000000005c
:10552800415f8000305f8000d04d8800000202009b
:1055380000000000a55780000500e00010003200c0
:1055480061836a000b00320062836a000600320041
:1055580063836a00010032003000370073b523000e
:10556800c23520000800370063d02300a22126009e
:105578000500370073ea230002aa2f000200370053
:105588001305240082942f00560202000000000038
:1055980011588800205888004358800052588000cd
:1055a80042030200000000003a29af00040037005f
:1055b800c3e92300f2eb20005602020000000000bd
:1055c800e1488800f0488800fe030200000000005f
:1055d80030588800e1488000f04880006358800017
:1055e8007258800061588800705888004203020091
:1055f800000000008324240002002000560202005c
:10560800000000002149880031498800fe0302009b
:1056180000000000105a8800000006000000060084
:105628000a68a80000000600082cef00082cec000f
:10563800b6027800f700200087836200871c780094
:10564800e70220000728e70007003700c70220000c
:105658000728e70004003700576080000638e60096
:1056680001003700f1ff37008024eb00082ced0023
:10567800000006000a88a900f20ba900082cef0018
:10568800082cec00b6027800f7002000878362003f
:10569800871c7800e70220000728e7000a00370087
:1056a800d70220000728e7000a000700c7022000e9
:1056b8000728e7000b003700576080000638e6002f
:1056c80001003700eeff37008024eb00082ced00c6
:1056d80000000600f20ba800082ced00a9027800d3
:1056e800000006000a88a80000000600082cec004c
:1056f800b6027800f700200087836200871c7800d4
:10570800c70220000728e700040037005760800020
:105718000638e60001003700f4ff37008024eb006c
:10572800082ced0000000600d2f1070049c1200056
:1057380039037800f500200005036300a65f8800a0
:1057480039037800f500200005036300b65f880080
:1057580039037800f500200005036300c65f880060
:1057680039037800f500200005036300d65f880040
:1057780039037800c8bf20000300080003000000b8
:1057880039037800f500200005036300061c780043
:10579800f20ba90066618000350520000628e700a5
:1057a800f20ba80070002000be0e020000000000ee
:1057b800405f800090658800305f800080658800c9
:1057c800acf1070009c3200039037800f500200078
:1057d80005036300a65f880039037800f500200000
:1057e80005036300b65f880039037800f5002000e0
:1057f80005036300c65f880039037800f5002000c0
:1058080005036300d65f880039037800f50020009f
:1058180005036300e65f880039037800e8bf2000cd
:10582800030008000300000039037800f500200099
:1058380005036300061c7800f20ba900566280007d
:10584800550420000628e700f20ba800800020007d
:10585800be0e020000000000405f8000b0658800b6
:10586800305f8000a06588000000060081f1070015
:10587800a6608000f500200005036300a65f88008d
:10588800b6608000f500200005036300b65f88005d
:10589800f20ba90010002000be0e0200000000005c
:1058a800415f8000305f80000002020000000000bd
:1058b80011658800006588006ef1070089c1200025
:1058c80039037800f500200005036300a65f88000f
:1058d80039037800f500200005036300b65f8800ef
:1058e8003903780088bf2000050008000300000085
:1058f80039037800f500200005036300061c7800d2
:10590800f20ba90070002000be0e0200000000008b
:10591800415f8000305f800000020200000000004c
:1059280043c62400021c2e00be0202000000000034
:105938001365800002658000440302000000000037
:10594800e3c8230052a32f00560202000000000003
:1059580001f0a00066618000e50420000628e70049
:1059680001f0a100516588004065880041f10700f9
:1059780086618000f500200005036300a65f8800ab
:1059880096618000f500200005036300b65f88007b
:10599800a6618000f500200005036300c65f88004b
:1059a800f20ba90020002000be0e0200000000003b
:1059b800415f8000305f80000002020000000000ac
:1059c80011658800006588002af1070069c3200076
:1059d80039037800f500200005036300a65f8800fe
:1059e80039037800f500200005036300b65f8800de
:1059f8003903780088bf2000050008000300000074
:105a080039037800f500200005036300061c7800c0
:105a1800f20ba90070002000be0e0200000000007a
:105a2800415f8000305f800000020200000000003b
:105a380043c62400021c2e00be0202000000000023
:105a48001365800002658000440302000000000026
:105a5800e3c8230052a32f005602020000000000f2
:105a680001f0a00056628000750520000628e700b6
:105a780001f0a100716588006065880000000600db
:105a8800b0598000010020000100e6000000060077
:105a9800a0598000310020000100e6000000060047
:105aa800842d02000000000040568000414a80001a
:105ab8000100e6000000060070658000705e880046
:105ac80060658000605e880050658000505e8800d8
:105ad80040658000405e880010588000405888006b
:105ae8002058800050588800e42aef00e22aef008e
:105af800e02aef003a09a8000b08a80000000600f9
:105b0800f00ae20001003a000600370080578000e2
:105b1800514a80000180e60002003700c82aec00e4
:105b280000000600c82aef0000000600516580004a
:105b380040658000335280002252800042030200f8
:105b480000000000e404020000000000030024003c
:105b58000001eb00be020200000000008101780095
:105b6800000178005602020000000000915c8800e5
:105b7800a05c88005165800040658000e804020050
:105b880000000000d15c8800e05c8800b15c8800ff
:105b9800c05c88003152800020528000e804020076
:105ba80000000000b35c8000c25c80005602020066
:105bb80000000000b15c8800c05c8800716580004e
:105bc8006065800053528000425280004203020008
:105bd80000000000e40402000000000003002400ac
:105be8000001eb00be020200000000008101780005
:105bf800000178005602020000000000b35c80003b
:105c0800c25c80005602020000000000935c800025
:105c1800a25c800044030200000000007a04020035
:105c280000000000ec040200000000000300240053
:105c38000001eb005602020000000000915c8800a1
:105c4800a05c88003a29af000300370023ac240089
:105c580062be240002003700f3b9240092d2250066
:105c68005602020000000000fe03020000000000cf
:105c78000152880010528800915c8000a05c80006e
:105c8800e404020000000000d35c8000e25c8000b5
:105c98005602020000000000b15c8800c05c880069
:105ca800915c8000a05c8000e80402000000000015
:105cb800915c8800a05c8800516580004065800088
:105cc800e404020000000000935c8000a25c8000f5
:105cd8005602020000000000915c8800a05c880069
:105ce8003152800020528000e404020000000000cd
:105cf800935c8000a25c8000420302000000000068
:105d0800b35c8000c25c8000be020200000000009c
:105d1800915c8800a05c880003f823000001eb0078
:105d28004403020000000000935c8000a25c800035
:105d380001f0a6000200370003f82b000001eb0079
:105d48008300780002007800f004020000000000e0
:105d5800915c8800a05c880051528000405280000d
:105d68007365800062658000420302000000000045
:105d7800e40402000000000001f0a6000b00370058
:105d8800915c8000a05c80002322240032982f00c0
:105d98005602020000000000f15c8800005d8800e7
:105da800fe0302000000000010003700910c2400e0
:105db800b0fd2000935c8000a25c800042030200da
:105dc80000000000915c8800a05c88002322240069
:105dd80032982f005602020000000000f15c880093
:105de800005d8800fe03020000000000f2578000fa
:105df800020050000110200000f0a6008000eb0017
:105e080001004000f0518800000006005165800044
:105e180040658000535e8000425e800042030200bd
:105e280000000000e4040200000000000300240059
:105e38000001eb00be0202000000000081017800b2
:105e4800000178005602020000000000915c880002
:105e5800a05c88005165800040658000e80402006d
:105e680000000000d15c8800e05c8800b15c88001c
:105e7800c05c8800515e8000405e8000e80402003b
:105e880000000000b35c8000c25c80005602020083
:105e980000000000b15c8800c05c8800716580006b
:105ea80060658000735e8000625e800042030200cd
:105eb80000000000e40402000000000003002400c9
:105ec8000001eb00be020200000000008101780022
:105ed800000178005602020000000000b35c800058
:105ee800c25c80005602020000000000935c800043
:105ef800a25c800044030200000000007a04020053
:105f080000000000ec040200000000000300240070
:105f18000001eb005602020000000000915c8800be
:105f2800a05c88003a29af000300370023ac2400a6
:105f380062be240002003700f3b9240092d2250083
:105f48005602020000000000fe03020000000000ec
:105f5800d1598800e0598800915c8000a05c8000dd
:105f6800e404020000000000d35c8000e25c8000d2
:105f78005602020000000000b15c8800c05c880086
:105f8800915c8000a05c8000e80402000000000032
:105f9800915c8800a05c88005165800040658000a5
:105fa800e404020000000000935c8000a25c800012
:105fb8005602020000000000915c8800a05c880086
:105fc800515e8000405e8000e40402000000000092
:105fd800935c8000a25c8000420302000000000085
:105fe800b35c8000c25c8000be02020000000000ba
:105ff800915c8800a05c880003f823000001eb0096
:106008004403020000000000935c8000a25c800052
:1060180001f0a6000200370003f82b000001eb0096
:106028008300780002007800f004020000000000fd
:10603800915c8800a05c8800715e8000605e8000d2
:106048007365800062658000420302000000000062
:10605800e40402000000000001f0a6000b00370075
:10606800915c8000a05c80002322240032982f00dd
:10607800560202000000000061598800705988002b
:10608800fe0302000000000010003700910c2400fd
:10609800b0fd2000935c8000a25c800042030200f7
:1060a80000000000915c8800a05c88002322240086
:1060b80032982f0056020200000000006159880043
:1060c80070598800fe03020000000000f2578000ab
:1060d800020050000110200000f0a6008000eb0034
:1060e800010040005059880000000600000006002a
:1060f8005165800040658000a3c52400920e2900e8
:106108005602020000000000fe030200000000002a
:10611800d1658800c0658800716580006065800071
:10612800a3c52400920e29005602020000000000b8
:10613800fe03020000000000f1658800e0658800a9
:10614800715e8000605e8000a3c52400920e290065
:106158005602020000000000fe03020000000000da
:10616800b15e8800a05e8800515e8000405e8000bd
:10617800a3c52400920e2900560202000000000068
:10618800fe03020000000000915e8800805e880027
:10619800000006008445880095458800a6458800cb
:1061a8000b68ae001e0037007460800085cd2000ab
:1061b8000428e70013003700b5118000051a78009d
:1061c80074608800a600200006a8e70007003700d2
:1061d8000b48a8000b68aa0084cd20000b68ae000d
:1061e80084de2000746088002b003700c6d82000a9
:1061f80004b0e6002800370084cd200074608800d1
:1062080025003700b51180004602200006a8e700e7
:1062180021003700051a7800746088001e003700d6
:106228007460800085de20000428e7001300370032
:10623800b5118000051a780074608800a600200057
:1062480006a8e700070037000b48a8000b68aa005b
:1062580084cd20000b68ae0084de200074608800c6
:106268000d003700c6e9200004b0e6000a00370038
:1062780084de20007460880007003700b5118000b4
:106288004602200006a8e70003003700051a780038
:1062980074608800000037003202af00c0ff37008a
:1062a8008445800095458000a64580003222a900db
:1062b80087c0a900004006008460a90000400600cd
:1062c80000a0fe00849fbe00869fbe00889fbe007f
:1062d8008a9fbe008c9fbe00bb0180003b5d88008a
:1062e800cb0180004b5d8800db0180005b5d88008e
:1062f800eb0180006b5d8800fb0180007b5d8800fe
:106308000b0280008b5d88000060fe003849af00fa
:10631800d1a2aa000b28aa000b28af00270037003b
:106328001828ec00c0408000910020000100e60021
:10633800210037001828ef006369af001a28ec0025
:106348006369ae001a28ed00d04080008107200064
:106358000180e6006369a90081f82f000100e600ca
:106368006369a800d040880002003b0001102000ab
:1063780000804000e05788006389af001c28ec00cb
:106388006389ae001c28ed00e0408000a1052000d4
:106398000180e6006389a90061fa2f000100e60088
:1063a8006389a800e040880002003b00010021004a
:1063b80000804000d0578800bb003700cc11020095
:1063c80000000000de2aec00fa5680004b06200090
:1063d8000bd0e7006c003700de2aef00e02aec0063
:1063e8000a578000cb0320000bd0e70008003700d5
:1063f800e02aef00e22aec001a578000cb032000c5
:106408000bd0e70002003700e22aef00e42aec0094
:106418000b08af005c003700e40ae2005a003a00bb
:10642800e20ae20058003a003a0020000b578000c8
:106438000b50e700420037004a0020000b5780004d
:106448000b50e7003c0037005a0020000b57800033
:106458000b50e700180037006a0020000b57800037
:106468000b50e700240037007a0020000b5780000b
:106478000bd0e700440037003849af000c48a800ab
:106488003849a9000c48ae003f0037008420a90015
:106498009420a90084a0a90094a0a90088a0a9001c
:1064a80098a0a90088c0a90098c0a90088e0a90000
:1064b80098e0a900340037003342a800010020000a
:1064c80091018800a115240033000800060000008f
:1064d8000000eb003140ba003302ae00feff370087
:1064e8000a00090000000000a01188003302ae0075
:1064f800feff3700920037003342a8000100200059
:1065080091018800211a24001100080006000000eb
:106518000000eb003140ba003302ae00feff370046
:106528000a00090000000000a01188003302ae0034
:10653800feff37008200370000042000c0118800e9
:106548003342a8000100200091018800e1182400ce
:1065580013000800060000000000eb003140ba00fc
:106568003302ae00feff37000a00090000000000f9
:10657800a01188003302ae00feff3700a002200001
:10658800c01188006e0037000b08af0023003700e9
:10659800e40ae20021003a00e20ae2001f003a00a1
:1065a80082002000035780000218e6002000370010
:1065b800c2012000035780000298e6001700370048
:1065c8008000eb003048800000020200000000005c
:1065d800a1488800b0488800814880009048800021
:1065e800833424000200200056020200000000004c
:1065f800a3488000b2488000440302000000000065
:106608009334240002002000be02020000000000b3
:106618008148880090488800050037000a13020066
:10662800000000008000eb003048800067f8070099
:1066380010418000110020000180e70002003700af
:106648008e09af0039fd07001041800021002000ad
:106658000180e700020037000b08af00ebfd0700e0
:1066680010418000310020000180e700050037005c
:10667800c04c8000110020000180e600620f02007b
:106688000000000010418000410020000180e70068
:106698000000370010418000510020000100e60092
:1066a8002228ec00260037000ae8ae001100370067
:1066b8003229ef0017fb070057fb07008cfe070085
:1066c8008000eb00f047800037f80700104888008a
:1066d8008000eb000048800033f80700204888005d
:1066e8006423020000000000622302000000000092
:1066f8000ae8a9000ac8ae000a0037002228ef00fd
:106708008628020000000000dafa070057fc07009c
:106718007cfb070070fb07000b08ae00d8fc0700e5
:106728000ac8a9000b88ae00050037003229ef001f
:1067380066fa07009af90700b8f907000b88a9005c
:10674800b23f020000000000ce130200000000006b
:106758005a15020000000000fa3e02000000000086
:1067680040418000c34c8000320020000218e7003e
:106778003058880030418000c34c8000320020002f
:106788000218e700505988000b48af004227020062
:10679800000000000b48a9005b5d8000db01880059
:1067a8006b5d8000eb0188007b5d8000fb01880049
:1067b8008b5d80000b0288008400a9008780a900f7
:1067c8004f06be004f05be004f04be004f03be007b
:1067d8004f02be000080fe00004006009780a9001e
:1067e80097c0a90060458800714588002342a80029
:1067f8000a00fc0080408000a10420000180e6001f
:106808004e003700000078004c00330000600100a3
:106818004a003700520037005a0037006700370037
:1068280074003700810037008e0037009b00370066
:10683800a8003700b5003700c2003700cf00370086
:10684800dc003700e9003700f600370003013700a5
:10685800100137001d0137002a01370037013700c2
:1068680044013700510137005e0137006b013700e2
:106878007801370085013700920137009f01370002
:10688800ac013700b9013700c6013700d301370022
:10689800db013700e3013700eb013700f301370074
:1068a800fb01370003023700100237001d023700d2
:1068b8002a023700370237003e0237004b02370002
:1068c8005802370064023700710237007e02370031
:1068d8008b02370098023700a5023700b202370052
:1068e800bf023700cc023700d9023700e602370072
:1068f800f3023700000337000d0337001903370090
:1069080025033700310337003d03370049033700bb
:1069180055033700610337006d03370079033700eb
:1069280085033700910337009d033700a90337001b
:10693800b5033700c1033700cd033700804080001e
:10694800201188000057800020118800105780000f
:10695800201188002057800020118800c4033700c8
:106968008040800020118800c057800020118800d6
:10697800e057800020118800f0578000201188001f
:10698800bb03370080408000201188003058800009
:10699800f10f20000080600020118800305880002e
:1069a80001f02f00008060000080fd0020118800a9
:1069b800d042800020118800ad033700804080005d
:1069c80020118800e0658000f10f20000080600041
:1069d80020118800e065800001f02f000080600031
:1069e8000080fd0020118800c05980002011880017
:1069f8009f0337008040800020118800f0658000e8
:106a0800f10f20000080600020118800f0658000f0
:106a180001f02f00008060000080fd002011880038
:106a2800a059800020118800910337008040800021
:106a380020118800c0658000f10f200000806000f0
:106a480020118800c065800001f02f0000806000e0
:106a58000080fd0020118800b059800020118800b6
:106a6800830337008040800020118800d0658000b3
:106a7800f10f20000080600020118800d0658000a0
:106a880001f02f00008060000080fd0020118800c8
:106a9800505980002011880075033700804080001d
:106aa80020118800805e8000f10f200000806000c7
:106ab80020118800805e800001f02f0000806000b7
:106ac8000080fd0020118800d04980002011880036
:106ad800670337008040800020118800905e8000a6
:106ae800f10f20000080600020118800905e800077
:106af80001f02f00008060000080fd002011880058
:106b080040568000201188005903370080408000db
:106b180020118800a05e8000f10f20000080600036
:106b280020118800a05e800001f02f000080600026
:106b38000080fd0020118800c04a800020118800d4
:106b48004b0337008040800020118800b05e800031
:106b5800f10f20000080600020118800b05e8000e6
:106b680001f02f00008060000080fd0020118800e7
:106b7800b0428000201188003d033700804080002b
:106b88002011880010488000f10f2000008060006c
:106b9800201188001048800001f02f00008060005c
:106ba8000080fd0020118800c0428000201188006c
:106bb8002f0337008040800020118800e0598000b2
:106bc800f10f20000080600020118800e05980004b
:106bd80001f02f00008060000080fd002011880077
:106be800d04a8000201188002103370080408000af
:106bf8002011880090598000f10f2000008060006b
:106c0800201188009059800001f02f00008060005a
:106c18000080fd0020118800e04a800020118800d3
:106c2800130337008040800020118800005880003e
:106c3800f10f2000008060002011880000588000bb
:106c480001f02f00008060000080fd002011880006
:106c5800b04a80002011880005033700804080007a
:106c68002011880040488000f10f2000008060005b
:106c7800201188004048800001f02f00008060004b
:106c88000080fd0020118800c05580002011880078
:106c9800f7023700804080002011880020488000db
:106ca800f10f20000080600020118800204880003b
:106cb80001f02f00008060000080fd002011880096
:106cc800e055800020118800e902370080408000ec
:106cd8002011880070578000f10f200000806000ac
:106ce800201188007057800001f02f00008060009c
:106cf8000080fd0020118800d055800020118800f8
:106d0800db02370080408000201188006057800037
:106d1800f10f20000080600020118800605780007b
:106d280001f02f00008060000080fd002011880025
:106d3800b055800020118800cd02370080408000c7
:106d48002011880080578000f10f2000008060002b
:106d5800201188008057800001f02f00008060001b
:106d68000080fd00201188009057800020118800c5
:106d7800bf02370080408000201188003043800027
:106d8800f10f20000080600020118800304380004f
:106d980001f02f00008060000080fd0020118800b5
:106da800004a800020118800b1023700804080002e
:106db8002011880050488000f10f200000806000fa
:106dc800201188005048800001f02f0000806000ea
:106dd8000080fd0020118800304a800020118800c2
:106de800a30237008040800020118800d05980001d
:106df800f10f20000080600020118800d059800029
:106e080001f02f00008060000080fd002011880044
:106e1800204a8000201188009502370080408000b9
:106e280020118800f0598000f10f200000806000d8
:106e380020118800f059800001f02f0000806000c8
:106e48000080fd0020118800f04980002011880092
:106e5800870237008040800020118800005a800097
:106e6800f10f20000080600020118800005a800087
:106e780001f02f00008060000080fd0020118800d4
:106e8800104a800020118800790237008040800075
:106e98002011880080588000f10f200000806000d9
:106ea800201188008058800001f02f0000806000c9
:106eb8000080fd0020118800404a800020118800d1
:106ec8006b0237008040800020118800504a800003
:106ed800f10f20000080600020118800504a8000d7
:106ee80001f02f00008060000080fd002011880064
:106ef800e0498000201188005d0237008040800052
:106f080020118800105a8000f10f200000806000d6
:106f180020118800105a800001f02f0000806000c6
:106f28000080fd0020118800c049800020118800e1
:106f38004f0237008040800020118800c047800041
:106f4800f10f20000080600020118800c0478000f9
:106f580001f02f00008060000080fd0020118800f3
:106f6800f04a8000201188004102370080408000ec
:106f780020118800d0478000f10f200000806000b9
:106f880020118800d047800001f02f0000806000a9
:106f98000080fd0020118800104b8000201188001f
:106fa800330237008040800020118800e0478000cd
:106fb800f10f20000080600020118800e047800069
:106fc80001f02f00008060000080fd002011880083
:106fd800304b800020118800250237008040800057
:106fe80020118800404b800020118800504b800001
:106ff80020118800604b8000201188001c02370097
:107008008040800020118800f05580002011880001
:10701800005680002011880010568000201188003a
:10702800130237008040800020118800205680001d
:1070380020118800204b800020118800a04b800080
:10704800201188000a023700804080002011880043
:107058008049800020118800b04b800020118800f2
:10706800c04b80002011880001023700804080005a
:1070780020118800204480002011880030448000be
:10708800201188005044800020118800f801370042
:107098008040800020118800404480002011880032
:1070a8003056800020118800104c80002011880084
:1070b800ef01370080408000201188005043800095
:1070c800f10f2000008060002011880050438000ec
:1070d80001f02f00008060000080fd002011880072
:1070e800204c800020118800e1013700804080009a
:1070f80020118800a0438000f10f2000008060006c
:1071080020118800a043800001f02f00008060005b
:107118000080fd0020118800304c8000201188007c
:10712800d30137008040800020118800b0438000e0
:10713800f10f20000080600020118800b04380001b
:1071480001f02f00008060000080fd002011880001
:10715800404c800020118800c50137008040800025
:1071680020118800c0438000f10f200000806000db
:1071780020118800c043800001f02f0000806000cb
:107188000080fd0020118800504c800020118800ec
:10719800b70137008040800020118800604c8000d3
:1071a80020118800c051800020118800201188001b
:1071b800af0137008040800020118800804c80009b
:1071c800f10f20000080600020118800804c8000b2
:1071d80001f02f00008060000080fd002011880071
:1071e800d051800020118800a10137008040800024
:1071f80020118800904c8000f10f20000080600072
:1072080020118800904c800001f02f000080600061
:107218000080fd0020118800e051800020118800c6
:10722800930137008040800020118800a04c800026
:10723800f10f20000080600020118800a04c800021
:1072480001f02f00008060000080fd002011880000
:1072580020118800860137008040800020118800b6
:10726800b04c8000f10f20000080600020118800e1
:10727800b04c800001f02f00008060000080fd000d
:1072880020118800704c8000201188007801370098
:10729800804080002011880000528000f10f2000fb
:1072a80000806000201188000052800001f02f004b
:1072b800008060000080fd0020118800f0518000ef
:1072c800201188006a013700804080002011880062
:1072d80010528000f10f200000806000201188000b
:1072e8001052800001f02f00008060000080fd0037
:1072f80020118800c04c8000201188005c013700f4
:107308008040800020118800905b8000f10f2000f1
:107318000080600020118800905b800001f02f0041
:10732800008060000080fd0020118800604180001e
:10733800201188004e01370080408000201188000d
:10734800a05b8000f10f2000008060002011880001
:10735800a05b800001f02f00008060000080fd002d
:1073680020118800704180002011880040013700fa
:107378008040800020118800b05b8000f10f200061
:107388000080600020118800b05b800001f02f00b1
:10739800008060000080fd0020118800904180007e
:1073a80020118800320137008040800020118800b9
:1073b800c05b8000f10f2000008060002011880071
:1073c800c05b800001f02f00008060000080fd009d
:1073d80020118800b0418000201188002401370066
:1073e8008040800020118800d0578000f10f2000d5
:1073f8000080600020118800d057800001f02f0025
:10740800008060000080fd0020118800404280005c
:107418002011880016013700804080002011880064
:10742800d04d8000f10f20000080600020118800fe
:10743800d04d800001f02f00008060000080fd002a
:1074480020118800d04c80002011880008013700e6
:107458008040800020118800e04d8000f10f20005e
:107468000080600020118800e04d800001f02f00ae
:10747800008060000080fd0020118800e04c800042
:1074880020118800fa003700804080002011880011
:10749800f04d8000f10f200000806000201188006e
:1074a800f04d800001f02f00008060000080fd009a
:1074b80020118800204d800020118800ec00370042
:1074c8008040800020118800004e8000f10f2000cd
:1074d8000080600020118800004e800001f02f001d
:1074e800008060000080fd0020118800504280006c
:1074f80020118800de0037008040800020118800bd
:10750800104e8000f10f20000080600020118800dc
:10751800104e800001f02f00008060000080fd0008
:10752800201188006042800020118800d0003700b8
:107538008040800020118800204e8000f10f20003c
:107548000080600020118800204e800001f02f008c
:10755800008060000080fd00201188002011880054
:10756800c30037008040800020118800304e800022
:10757800f10f20000080600020118800304e80004c
:1075880001f02f00008060000080fd0020118800bd
:1075980020118800b6003700804080002011880044
:1075a800404e8000f10f200000806000201188000c
:1075b800404e800001f02f00008060000080fd0038
:1075c8002011880020118800a90037008040800021
:1075d80020118800504e8000f10f200000806000cc
:1075e80020118800504e800001f02f0000806000bc
:1075f8000080fd0020118800201188009c003700c1
:107608008040800020118800604e8000f10f20002b
:107618000080600020118800604e800001f02f007b
:10762800008060000080fd00201188002011880083
:107638008f0037008040800020118800704e800045
:10764800f10f20000080600020118800704e80003b
:1076580001f02f00008060000080fd0020118800ec
:1076680020118800820037008040800020118800a7
:10767800804e8000f10f20000080600020118800fb
:10768800804e800001f02f00008060000080fd0027
:107698002011880020118800750037008040800084
:1076a80020118800904e8000f10f200000806000bb
:1076b80020118800904e800001f02f0000806000ab
:1076c8000080fd0020118800201188006800370024
:1076d8008040800020118800a04e8000f10f20001b
:1076e8000080600020118800a04e800001f02f006b
:1076f800008060000080fd002011880020118800b3
:107708005b0037008040800020118800b04e800068
:10771800f10f20000080600020118800b04e80002a
:1077280001f02f00008060000080fd00201188001b
:10773800201188004e00370080408000201188000a
:10774800c04e8000f10f20000080600020118800ea
:10775800c04e800001f02f00008060000080fd0016
:1077680020118800201188004100370080408000e7
:1077780020118800d04e8000f10f200000806000aa
:1077880020118800d04e800001f02f00008060009a
:107798000080fd0020118800201188003400370087
:1077a8008040800020118800e04e8000f10f20000a
:1077b8000080600020118800e04e800001f02f005a
:1077c800008060000080fd002011880020118800e2
:1077d800270037008040800020118800f04e80008c
:1077e800f10f20000080600020118800f04e80001a
:1077f80001f02f00008060000080fd00201188004b
:10780800201188001a00370080408000201188006d
:10781800004f8000f10f20000080600020118800d8
:10782800004f800001f02f00008060000080fd0004
:1078380020118800201188000d003700804080004a
:1078480020118800104f8000f10f20000080600098
:1078580020118800104f800001f02f000080600088
:107868000080fd00201188002011880000003700ea
:107878001028ec0081408000a00420000088e60069
:107888001028ef00604580007145800097c0a8006f
:107898008400a9009780a800004006007746880069
:1078a8008846880099468800d502af001000370046
:1078b800070a8000884480000838e6000300370083
:1078c800888353007744880004003700490d23005b
:1078d8000884540087034400774488007746800072
:1078e80088468000994680008420a9000040060050
:1078f800070a80004261af00fdff37008744880017
:107908007746800088468000994680008420a90038
:1079180000400600b7468800c8468800d946880057
:10792800d522af0010003700270a8000a844800045
:107938000838e6000300370088835300974488001e
:1079480004003700490d23000884540087034400cd
:1079580097448800b7468000c8468000d946800012
:1079680084a0a90000400600270a80004661af00f5
:10797800fdff3700a7448800b7468000c84680004e
:10798800d946800084a0a90000400600f746880078
:107998000847880019478800d542af002000370003
:1079a800470a8000c84480000838e6000b0037000a
:1079b80088835300b74488006289ae0013003700fb
:1079c8003849a900084c800008b8e6003849a800e2
:1079d8000c48af003849a9000c003700490d2300b6
:1079e8000884540087034400b74488006289ae00c5
:1079f800060037003849a900084c800008b8e6009e
:107a08003849a8000c48af003849a900f74680005b
:107a1800084780001947800088a0a9000040060098
:107a2800470a80004a61af00fdff3700c74488005d
:107a3800f7468000084780001947800088a0a90001
:107a480000400600274788003847880049478800d3
:107a5800d562af0010003700670a8000e844800054
:107a68000838e6000300370088835300d7448800ad
:107a780004003700490d230008845400870344009c
:107a8800d74488002747800038478000494780004e
:107a980088c0a90000400600670a80004e61af0058
:107aa800fdff3700e74488002747800038478000fb
:107ab8004947800088c0a900004006005747880051
:107ac8006847880079478800d482af002e003700c5
:107ad800870a8000084580000838e6000300370060
:107ae80088835300f744880004003700490d2300b9
:107af8000884540087034400f74488003821200094
:107b080008b8e600060037006289ae003849a800c8
:107b18000c48af003849a9003429ef001500370098
:107b2800f85520000838e600060037006289ae00e4
:107b38003849a8000c48af003849a9003429ef009b
:107b48000c0037003429ec00a8498000a700200069
:107b58006289af000200370007c0e6003849a90073
:107b680007c0e6003429ef000c48af003849a900e7
:107b78002221ef005747800068478000794780003e
:107b880088e0a90000400600870a80005261af0023
:107b9800fdff370007458800574780006847800089
:107ba8007947800088e0a90000400600b7458800b2
:107bb800c8458800d94588000c08af000b0037007d
:107bc8000be8a9000c08a8006228ef006428ef0061
:107bd8005641a9005621a8005601a800a70a80000e
:107be8005661af00f1ff370039003700a70a80005f
:107bf800480d230008b8e60027003700c8ce220049
:107c080008b8e6002c0037000be8ae002200370069
:107c1800c851220008b8e6001f00370048132200a8
:107c280008b8e600130037004896210008b8e600b7
:107c380019003700c85721000838e6001600370039
:107c48006428ec006228d7006368a900c8002000f7
:107c58002943800009c0e7001b0037001843800053
:107c6800384388002fe1a8009900a9000c28a80033
:107c7800090037006428ec006228d7006368a80070
:107c8800c80020002943800009c0e7000e00370023
:107c980018438000384388000c08a9000be8a900a5
:107ca8006228ef006428ef005641a9005621a80079
:107cb8005601a900060037000c08a8000be8a80028
:107cc8006228ef006428ef005661af00b7ff370065
:107cd80013e1a9008500a9000a21ef0013e1a8001b
:107ce800b7458000c8458000d94580008900a900b3
:107cf800004006006446880024002000540c8800d8
:107d0800644680008440a90000400600a44688001c
:107d180024002000840c8800a446800084c0a900a8
:107d280000400600e446880024002000b40c8800c7
:107d3800e44680008720a900004006008740a9008b
:107d4800004006001546880065498000750c8800cb
:107d580075498000a50c880045498000150c8800ed
:107d680055498000450c880025002000250c880016
:107d78001546800084e0a900004006000c28ae00eb
:107d8800070037000c28a9006628ef002fe1a9009a
:107d98008a00a9002621ef002fe1a8000040060074
:107da8002fe1a9008a00a9002621ef008900a90077
:107db8009900a800004006003429ef006289ae004f
:107dc8003849a8000c48af003849a90089e0a90043
:107dd8000040060021e3a9002043a9008de3a90083
:107de80085c0a90085a0a900004006000500240060
:107df800b5017800c2568000440120000410b90083
:107e0800030040000180b000530120001100090068
:107e18004308d800c056880000488800b50178009b
:107e2800d2568000440120000410b900030040002d
:107e38000180b00053012000110009004308d80058
:107e4800d056880030488800b5017800724180001b
:107e5800440120000410b900030040000180b00074
:107e680053012000110009004308d8007041880020
:107e7800b5017800b2568000440120000410b90012
:107e8800030040000180b0005301200011000900e8
:107e98004308d800b0568800f0478800b50178003c
:107ea800924380007410b900030040000180b000c4
:107eb80053012000110009004308d80090438800ae
:107ec800d32620000300500080438800b5017800c5
:107ed80092418000440120000410b90003004000d2
:107ee8000180b00053012000110009004308d800a8
:107ef80090418800b5017800b50178007243800090
:107f08007410b900030040000180b0005301200044
:107f1800110009004308d8007043880060438800b6
:107f2800b5017800b5017800b5017800b24180004c
:107f3800440120000410b900030040000180b00093
:107f480053012000110009004308d800b0418800ff
:107f5800b501780085a0a9000000060070448000e3
:107f68003069af0010518000030120000300b90000
:107f780043062000110009004308d8002044880067
:107f880090448000030120000300b900430620004c
:107f9800110009004308d80030448800b04480002c
:107fa800030120000300b900430620001100090066
:107fb8004308d80040448800d04480003049af00ce
:107fc80040518000030120000300b900430620004f
:107fd800110009004308d80050448800f04480008c
:107fe800030120000300b900430620001100090026
:107ff8004308d80060448800000006000100200003
:1080080091018800018024001100ba00f2ff2f00be
:1080180002016800110032000043880002082000b5
:108028008100410002c024000288e700f6ff370003
:1080380002082000828050003100ba00a29320007c
:1080480035000800030000000000eb003100ba0012
:108058000019780000000000000006000208200057
:10806800828050003100ba00a29320003500080039
:10807800030000000000eb003100ba00001978008e
:1080880000000000000006000100200091018800a7
:10809800018024001100ba00f2ff2f0002016800dd
:1080a80015003200004388000208200081004100ca
:1080b80002c024000288e700f6ff370002402000d3
:1080c800828050001100ba000000e80000438800d8
:1080d8008c400200000000000243800010002400d1
:1080e800003b88000300200093018800ac40020098
:1080f800000000000000060010002400003b88007b
:1081080002438000ac4002000000000000000600ae
:1081180020042400003b880003002000930188000d
:108128008108bb000500fc0050052000303b88009a
:10813800a20a2000323b880061e7a8000000000086
:108148000000000061e7af00feff370000000600f6
:10815800020078008008bb008098bb00a293200032
:1081680035000800040000000000eb003200780031
:108178008008bb008098bb000000000000000000e1
:108188000500fc0050052000303b8800a10a2000b3
:10819800313b880061e7a8000000000000000000f3
:1081a80061e7af00feff3700000006000000000096
:1081b8000100000004000000070000000b000000a0
:1081c8000e0000001100000014000000170000005d
:1081d8001b0000001e000000210000002500000018
:1081e800280000002b0000002f00000033000000d2
:1081f800360000003a0000003e0000004200000087
:10820800460000004a0000004e0000005200000036
:10821800570000005b0000006000000065000000df
:108228006b00000070000000760000007c00000079
:1082380082000000880000008f0000009700000006
:108248009f000000a7000000af000000b900000078
:10825800c3000000ce000000da000000e7000000c4
:10826800f5000000040100001601000029010000cb
:108278003e0100005601000071010000910100005c
:10828800b7010000e3010000180200005a020000d4
:10829800ad0200001a030000af03000087040000cd
:1082a800e105000069080000270f000024500000c5
:1082b8004d5400004b330000313400002c300000d6
:1082c8002c3100002c3100002c3100002c30000033
:1082d8002c3000002c3000002c3000002c30000026
:1082e8002c3000002c3000002c3000002c30000016
:1082f8002c3000002c3000002c3000002c30000006
:108308002c3000002c3000002a320000390d00000b
:108318000a000000245000004d5400004b320000b9
:10832800353100002c3500003736000030300000b1
:108338002a320000430d00000a000000245000000b
:108348004d5400004b320000323000002c32000047
:10835800303000002a320000430d00000a000000ff
:10836800245000004d5400004b3500003030000010
:108378002c320000303000002c3000002c3000007f
:108388002c3000002c3000002a310000410d000084
:108398000a000000245000004d5400004b33000038
:1083a800303000002c320000303000002c3000004b
:1083b8002c3000002c3000002c3000002a31000046
:1083c800430d00000a00000024470000505600003a
:1083d800544700002c310000393800002e390000c5
:1083e800372c0000542c00002c4d00002c300000cd
:1083f8002e320000313300002c4e00002c300000db
:108408002e330000393400002c4b00002c410000b2
:108418002a330000440d00000a0000002447000031
:1084280050470000474100002c3000003131000067
:1084380035320000382e000030300000302c0000ab
:1084480031380000323700002e3100003931000089
:1084580030300000302c00004e2c00003036000078
:1084680039350000372e0000363600003030000065
:10847800303000002c5700002c3100002c37000051
:108488002c3000002e390000382c00002d3100005f
:10849800382e000033310000392c00004d2c00002c
:1084a800313700002e380000303600002c4d000017
:1084b8002c2c00002a360000460d00000a0000009f
:1084c80024470000505200004d4300002c300000ab
:1084d8003533000037340000302e00003030000003
:1084e800302c0000412c00003235000030330000f1
:1084f8002e36000033310000392c00004e2c0000cd
:108508003132000031330000362e000030300000d8
:10851800393900002c4500002c3200002e360000ae
:10852800392c0000373900002e360000352c0000a9
:108538003130000030310000303600002c2c0000b3
:108548002c4100002a350000330d00000a0000000d
:020000040000fa
:1085580000080000f806000000000000000000000d
:020000040000fa
:048568000000fe0011
:00000001FF
